:10000E00000000C0F0F87C7C7C7CF8F0C0000000A2
:10001E000000FCFF1F010000000001DFFFFE0000DA
:10002E0000FEFFFF0000C0E0F8FE3F0FFFFFFE00E6
:10003E00007FFFFFFC3F1F0701000000FFFF1F00B6
:10004E0000001FFFFCC080000080E0FCFF1F0000CE
:10005E0000000001070F0F1F1F0F07030000000015
:10006E0000000080C0E0F0F8FCFC00000000000082
:10007E0000000E1F0F0701FFFFFF00000000000031
:10008E0000000000000000FFFFFF00000000000065
:10009E0000000000000000FFFFFF00000000000055
:1000AE0000008080808080FFFFFF808080800000C5
:1000BE0000000F0F0F0F0F0F0F0F0F0F0F0F00007E
:1000CE00000080E0F0F87C7C7CFCF8E08000000012
:1000DE00000000070100000000000FFFFF000000FD
:1000EE00000000000000000000C0FEFF1F00000026
:1000FE00000000000080E0F8FE3F07010000000055
:10010E000000C0F0FCBF8F83808080808080000064
:10011E0000000F0F0F0F0F0F0F0F0F0F0F0F00001D
:10012E00000000F8787C7C7C7CF8F8E08000000011
:10013E0000000000000000000000FFFFFF000000B4
:10014E000000000000F0F0F0F0FCDF8F0100000076
:10015E000000000000010101010307FFFEF800008E
:10016E00000080800000000080C0E0FFFF0F000054
:10017E0000000F0F0F1F1F0F0F0F070100000000D1
:10018E0000000000000000C0F8F8F8F800000000C1
:10019E000000000000E0FE7F0700FFFF00000000EF
:1001AE00000080F0FF3F03000000FFFF0000000092
:1001BE0000F8FFDFC1C0C0C0C0C0FFFFC0C0C0009C
:1001CE0000070707070707070707FFFF07070700CF
:1001DE00000000000000000000000F0F00000000F3
:1001EE00000000F8F8787878787878787800000051
:1001FE00000000FFFF0000000000000000000000F3
:10020E00000000FFFFF8F8F8F8F0F0E080000000C2
:10021E000000000000000000000107FFFFFC0000CE
:10022E00000000800000000080C0F0FF7F0700008B
:10023E000000000F0F1F1F0F0F070301000000002B
:10024E000000000080C0E0F0F8F878787800000038
:10025E00000080FCFF0F0301000000000000000002
:10026E000000FFFFE1F0F8787C78F8F0E080000005
:10027E000000FFFF0100000000000007FFFF00006C
:10028E0000001FFFFFC080000000C0F0FF7F0000D5
:10029E0000000000030F0F1F1F0F0F0701000000CB
:1002AE000000F8F8F8F8F8F8F8F8F8F8F8F80000A0
:1002BE0000000000000000000000E0FF7F070000CB
:1002CE000000000000000000C0FEFF0F0000000054
:1002DE0000000000000080FCFF3F01000000000055
:1002EE000000000000F8FF7F030000000000000087
:1002FE00000000000F0F0F000000000000000000C3
:10030E00000000E0F0F87C7C7C7CF8F8E000000057
:10031E000000FFFFFF000000000000FFFFFF0000D5
:10032E000000010F1FFFFCF8F0FCFE1F070000008D
:10033E000000F0FCFF0F070103071FFFFEF0000097
:10034E000000FFFFF0C080000080C0F0FF7F0000C3
:10035E0000000003070F0F1F1F0F0F070300000001
:10036E00000000E0F0F87C3C7C7CF8F0800000009F
:10037E0000E0FFFF07000000000001FFFFF8000093
:10038E000003FFFFF08080008080C0E0FFFF0000D0
:10039E0000000003070F0F0F0F0707F3FFFF00000A
:1003AE0000000080808080C0E0F0FC7F0F00000025
:1003BE000000000F0F0F0F070703010000000000E1
:1003CE0000F03C0E0E1CF80000FFE0381C07FF7F0B
:1003DE00000F1C3030380F000070381CFE0000007B
:1003EE0000000000FF000000003838383F383800A9
:1003FE0000181C0E0EFCF000000000C0F03F0700BD
:10040E0000383E3B38383800000C0C0E0EFCF00065
:10041E0000001C1C1C3FE10000303030301C0F006F
:10042E00000000E03CFC0000C0F88F8180FF80805F
:10043E0001010101013F010100FCFC0C0C0C0C0040
:10044E00000F0F0C0C3CF00000303030381C070051
:10045E0000C0F01C0C0C0C0000FF1C0C0E0CF80065
:10046E0000071E3030380F00000C0C0C0CCCFC00BA
:10047E0000000080F80F00000000381F010000008F
:10048E0000F09C0E0E0CF80000C1771E1C7FE300DE
:10049E00001F383030381F0000F01C0E0E1CF0000C
:1004AE00001F38303018FF0000303038180E0300AF
:1004BE0000000000000000000000F03C0C0C0C00DE
:1004CE000000F03C0C0C0CFC03030303FC00000CBE
:1004DE000CFF0C0C0C00000C0CFF0C0C0C000F3065
:1004EE003030300F000000003F0000000000000020
:1004FE003F00000000C03030C000C030303030C08F
:10050E00030C0C0300FF00000000030000000000BD
:10051E000F303030300F00F00000000000F000000F
:10052E003FC000C03F000000000F300F0000000071
:10053E0000003C3CF00C030303030303030303031B
:10054E00030303030303030303030303030303036D
:10055E00030303030303030303030303030303035D
:10056E000303030303030303030CF00F30C0C0C0E7
:10057E00C0C0C0C0C0C0C0C0C0C0C0C0C0C0C0C06D
:10058E00C0C0C0C0C0C0C0C0C0C0C0C0C0C0C0C05D
:10059E00C0C0C0C0C0C0C0C0C0C0C0C0C0C0C0C04D
:1005AE00300F000CF00C0C0C300000000F3030300F
:1005BE000C0000FC0C0C0CF0000000FF0303030009
:1005CE000000C0F0FCFCFCFCFCFCFCFCFCFCFCFC9D
:1005DE00FCFCFCFCFCFCFCFCFCFCFCFCFCFCFCFC4D
:1005EE00FCFCFCFCFCFCFCFCFCFCF0C0FFFFFFFF79
:1005FE00FFFFFFFF00FFFFF3F3F3F3F3F3F3F3F368
:10060E00FFFFFFFFF30FFFFF03F3F3F3F3F303FF1C
:10061E00FFFFFFFFFFFFFFFFFFFFFFFF03FF00FCDA
:10062E00F3FF003C3C3C3C3C00FFFFFFFCC3FF3FA4
:10063E00FFFF003C3C3C3C3C00FFFFFFFFFFFFFF89
:10064E00FFFFFFFFFFFCFFFF00FFFFFF00CFCFCF3D
:10065E00CFCF00FFFFFFCFCF03FCFF03F3F303F376
:10066E0003F3F303FFFFFFFFFFFFFFFFFFFFFFFF9C
:10067E00FFFF00FFFFCFCFCFCFCFCFCFCFCFFFFF2B
:10068E00FFFFC0FFCFC0CFCFC0CFC0CFCFC0CFFFF7
:10069E00FFFFFFFF030F3F3F3F3F3F3F3F3F3F3FC8
:1006AE003F3F3F3F3F3F3F3F3F3F3F3F3F3F3F3F4C
:1006BE003F3F3F3F3F3F3F3F3F3F3F3F0F03C0F076
:1006CE00FCFCFCFCFCFCFCFCFCFCFCFCFCFCFCFC5C
:1006DE00FCFCFCFCFCFCFCFCFCFCFCFCFCFCFCFC4C
:1006EE00FCFCFCFCFCFCF0C0FFFFFFFFFFFFFFFF6C
:1006FE0000FFFFFFFFFF3F3F3F3F3FFFFFFF3F3F3B
:10070E003F003F3FFF3F3F003F3F3FFFFFFFFFFFE9
:10071E00FFFFFFFFFFFFFFFCFCFC00FCFC00FFFFE8
:10072E0000FFFFFF00FFFFFFFFFF3F00CFCFFFFFE8
:10073E00CF00FFFF00FFFFFFFFFFFFFFFFFFFFFFE9
:10074E00FFFFFFFF00FFFF00FFFF00FFFFFF00FFA7
:10075E00FFFFFCCC3FC0FFFF3FCFF0FFF0FFF0CF1D
:10076E0000FFFFFFFFFFFFFFFFFFFF3FCFF0FFCFB9
:10077E003FC0FFFFC0F3F3F3C0FFFFFF3FC3FFFF18
:10078E00F30FFFFFF30FFFFFF30FFFFFFFFFFFFF5F
:10079E00030F3F3F3F3F3F3F3F3F3F3F3F3F3F3FC7
:1007AE003F3F3F3F3F3F3F3F3F3F3F3F3F3F3F3F4B
:1007BE003F3F3F3F3F3F3F3F0F03C0300C0C0C0C01
:1007CE000C0C0C0C0C0C0C0C0C0C0C0C0C0C0C0C5B
:1007DE000C0C0C0C0C0C0C0C0C0C0C0C0C0C0C0C4B
:1007EE000C0C30C0FF0000000000000000033C00B5
:1007FE0000000000300F0000000000C0030C000CD1
:10080E000C0CCC0C0C0C0CFC0000000000FFFF00CC
:10081E000000000000000303030303FF03030303B0
:10082E000300000000FF000C0C0C0CCCFF0C0C0C99
:10083E0000FF0000000000FFFF00000000000303A7
:10084E0003030303F30FF30303030303030000FF88
:10085E0000C0300C0300FF00000000FF000000008D
:10086E0000FFFF0000000000C0C030300C0300008D
:10087E0000030C3030C0C00000FF00000000030C6D
:10088E0003000030C03F0000000000FF030C3030BA
:10089E00303030303030303030303030303030304A
:1008AE00303030303030303030303030303030303A
:1008BE00303030300C0300F0FCFCFFFFFFFFFFFF79
:1008CE00FFFFFFFFFFFFFFFFFFFFFFFFFFFFFFFF2A
:1008DE00FFFFFCFCF000FFFFFFFFFFFFFFFFFFFF2E
:1008EE00FFFFFFFFFFFFFFFFFFFFFFFFFFFFFFFF0A
:1008FE00FFFFFFFFFFFFFFFFFFFFFF3F3F3F3F3FBA
:10090E003FFFFF3F3F3F3F3FFF3F3F3F3F3F3FFFE9
:10091E00FFFFFFFFFFFFFFFFFFFFFFFF00FFFFFFD8
:10092E00FF00FFFFFF00FFFFFFFF00FFFFFFFFFCC9
:10093E0003FFFFFFFFFFFFFFFFFFFFFF00FCFCFCBD
:10094E00FCFFFFFFFF00FFFFFFFF00FFFFFFFFFFAA
:10095E0000FFFFFFFFFFFFFFFFFFFFF3F0F3FFFFBF
:10096E00FFFFFFF3F3F0F3F3FFF3F0F3F3F3F3FC16
:10097E00FFFFFFFFFFFFFFFFFFFFFFFFFFFFFFFF79
:10098E00FFFFFFFFFFFFFFFFFFFFFFFFFFFFFFFF69
:10099E00FFFFFFFFFFFF000F3F3FFFFFFFFFFFFFC8
:1009AE00FFFFFFFFFFFFFFFFFFFFFFFFFFFFFFFF49
:1009BE00FFFF3F3F0F0000F0FCFCFFFFFFFFFFFFBC
:1009CE00FFFFFFFFFFFFFFFFFFFFFFFFFFFFFFFF29
:1009DE00FFFFFCFCF000FFFFFFFFFFFFFFFFFFFF2D
:1009EE00FFFFFFFFFFFFFFFFFFFFFFFFFFFFFFFF09
:1009FE00FFFFFFFFFFFFFFFFFFCF3FFFFF03F3F3FD
:100A0E00F3F303FFFFFFFFFF3F3F3F3F330F3F3F38
:100A1E003F3F3FFFFFFFFFFFF3CFFFFFFF003C3CD9
:100A2E003C3C00FFFFFFFFFF00F3F3003333333393
:100A3E0000F3F3FFFFFFFFFFFF0FF0FF03F303F3DE
:100A4E00F303F303FFFFFFFF00FFF3C333F3F333AF
:100A5E00C3F3FFFFFFFFFFFFF0FFFFCFC0CFC0CFFD
:100A6E00CFC0CFC0CFFFCFF0FFCFCFF3F3FCFCF35F
:100A7E00F3CFCFFFFFFFFFFFFFFFFFFFFFFFFFFFE4
:100A8E00FFFFFFFFFFFFFFFFFFFFFFFFFFFFFFFF68
:100A9E00FFFFFFFFFFFF000F3F3FFFFFFFFFFFFFC7
:100AAE00FFFFFFFFFFFFFFFFFFFFFFFFFFFFFFFF48
:100ABE00FFFF3F3F0F0000F0FCFCFFFFFFFFFFFFBB
:100ACE00FFFFFFFFFFFFFFFFFFFFFFFFFFFFFFFF28
:100ADE00FFFFFCFCF000FFFFFFFFFFFFFFFFFFFF2C
:100AEE00FFFFFFFFFFFFFFFFFFFFFFFFFFFFFFFF08
:100AFE00FFFFFFFFFFFFFFFFFFFFFF03FFFF3F03B0
:100B0E003F3F3F033F3FFFFFFFFFFFFFFFFF03FF9F
:100B1E00F3CFFFFFFFFFFFFFFFFC3C003CFF033066
:100B2E003333333003FFFC3C3C3C3C3CFCFC00FCD0
:100B3E00FCFCFCFFFFFFFFFFFFF3FC00FF3C30332C
:100B4E0033033333303FFFFFFF00FFFFFFFFF00F94
:100B5E00FFFF3FFFFFFFFFFFFFFFFFC0FFCFCFF302
:100B6E00FCFFFCF3CFCFF3F3F3F0FCFCFCFFFFFF35
:100B7E00FCF3C0FFFFFFFFFFFFFFFFFFFFFFFFFFC5
:100B8E00FFFFFFFFFFFFFFFFFFFFFFFFFFFFFFFF67
:100B9E00FFFFFFFFFFFF000F3F3FFFFFFFFFFFFFC6
:100BAE00FFFFFFFFFFFFFFFFFFFFFFFFFFFFFFFF47
:100BBE00FFFF3F3F0F0000F0FCFCFFFFFFFFFFFFBA
:100BCE00FFFFFFFFFFFFFFFFFFFFFFFFFFFFFFFF27
:100BDE00FFFFFCFCF000FFFFFFFFFFFFFFFFFFFF2B
:100BEE00FFFFFFFFFFFFFFFFFFFFFFFFFFFFFFFF07
:100BFE00FFFFFFFFFFFFFFFFFFCF3FFFFF0FCFCF37
:100C0E00CFCF0FFFFFFFFF0FFFFFFFFF03FFFFFF22
:100C1E00FF0FFFFFFFFFFFFF3F3F3CFFFF00CC0C2E
:100C2E00CCCCC03FFFFFFFC0CFCFCFCF00CFCFCFB9
:100C3E00CFC0FFFFFFFFFFFFFFFF00FFFF003FCF13
:100C4E00FCF3CC3FFFFF03FFFFFFFFFF00FFFFFFA3
:100C5E00FFFF03FFFFFFFFFFCFF3FCF3CFCCCFCFA0
:100C6E00CFCFCFCCCFFFF0F3F3F3F3F3F0F3F3F3F7
:100C7E00F3F3C0FFFFFFFFFFFFFFFFFFFFFFFFFFCD
:100C8E00FFFFFFFFFFFFFFFFFFFFFFFFFFFFFFFF66
:100C9E00FFFFFFFFFFFF000F3F3FFFFFFFFFFFFFC5
:100CAE00FFFFFFFFFFFFFFFFFFFFFFFFFFFFFFFF46
:100CBE00FFFF3F3F0F00000000000000000000009B
:100CCE000000C0C0C0000000000000C0C0F0F0FC7A
:100CDE00FCFFFFFFFFFFFFFCC0FCFFFFFFFFFFFF5E
:100CEE00FFFFFFFFFFFFFFFFFF033FFFFFFFFFFFC2
:100CFE00FFFFFFFFFFFFFFFFFFFF000000000303EA
:100D0E000F0F3F3FFFFFFFFFFFFF3F000000000000
:100D1E000000000000000003030300000000C0C03C
:100D2E00C0000000000000000000000000FCFFFFFB
:100D3E00FFFFFFFFFCFCF0F0C0C000000000FFFF53
:100D4E00FFFFFFFFFFFFFFFFFFFFFFFFFFFCC0FFE7
:100D5E00FFFFFFFFFFFFFFFFFFFFFFFFFFFF3F0351
:100D6E003FFFFFFFFFFFFF3F3F0F0F03030000009A
:100D7E00000000030303000000000000000000005C
:100D8E000000000000000000000000000000C0C0D5
:100D9E00C0000000000000C0C0F0F0FCFCFF3F3FB0
:100DAE000FFFFFFCC0FCFFFF3F0F0F03030000000F
:100DBE000000FFFFFF033FFFFFFCF0F0C0C000008C
:100DCE00000000FFFFFF0000000003030F0F3F3F76
:100DDE00FFFCFCF0FFFF3F000000000000000000E1
:100DEE00000000030303000000000030CCFCFCCC2C
:100DFE003000000030CCFCFCFCFCFCFCFCFCCC30DD
:100E0E000000C0C0C0000000000000000000000094
:100E1E0000FCFFFF0F3F3FFFFCFCF0F0C0C00000E6
:100E2E000000FFFFFF000000000003030F0F3FFF55
:100E3E00FFFCC0FFFFFF0000000000C0C0F0F0FC90
:100E4E00FFFF3F033FFFFFF0FCFCFF3F3F0F0F0391
:100E5E000300000000000003030300000000000078
:100E6E0000000000000000F0FCFCFFFFFFFFFFFF92
:100E7E00FFFFFFFFFFFFFFFFFFFFFFFFFFFFFCFC7A
:100E8E00F000FFFFFFFFFFFFFFFFFFFFFFFFFFFF72
:100E9E00FFFFFFFFFFFFFFFFFFFFFFFFFFFFFFFF54
:100EAE00FFFFFFFF00FFFF3FCFF3FCFFFF00FCFC47
:100EBE00FCFCF30FFFFFFFFFFFFFFFFFFFFFFFFF36
:100ECE0000F3CC3FFFFFFFFFFF00CFCFCFCFF3FCF0
:100EDE00FFFFFFFFFFFFFFFFFFFFFFFFC0FFFFFF53
:100EEE00FCF3CFFFFFC0FFFFFFFFFFFFFFFFFFFF82
:100EFE00FFFFFFFFFFFFFFFFFFFFFFFFFFFFFFFFF4
:100F0E00FFFFFFFFFFFFFFFFFFFFFFFFFFFF000FD2
:100F1E003F3FFFFFFFFFFFFFFFFFFFFFFFFFFFFF53
:100F2E00FFFFFFFFFFFF3F3F0F0000F0FCFCFFFF46
:100F3E00FFFFFFFFFFFFFFFFFFFFFFFFFFFFFFFFB3
:100F4E00FFFFFCFCF000FFFFFFFFFFFFFFFFFFFFB7
:100F5E00FFFFFFFFFFFFFFFFFFFFFFFFFFFFFFFF93
:100F6E00FFFFFFFFFFFFFFFF00FFFF3FCFF3FCFF81
:100F7E00FFFCFCFC00FCFCFCFFFFFFFFFFFFFFFF84
:100F8E00FFFFFFFF00F3CC3FFFFFFFFFFFFFFFFF61
:100F9E0000FFFFFFFFFFFFFFFFFFFFFFFFFFFFFF52
:100FAE00C0FFFFFFFCF3CFFFFFCFCFCFC0CFCFCF20
:100FBE00FFFFFFFFFFFFFFFFFFFFFFFFFFFFFFFF33
:100FCE00FFFFFFFFFFFFFFFFFFFFFFFFFFFFFFFF23
:100FDE00FFFF000F3F3FFFFFFFFFFFFFFFFFFFFF82
:100FEE00FFFFFFFFFFFFFFFFFFFF3F3F0F0000F080
:100FFE00FCFCFFFFFFFFFFFFFFFFFFFFFFFFFFFFF9
:10100E00FFFFFFFFFFFFFCFCF000FFFFFFFFFFFFF6
:10101E00FFFFFFFFFFFFFFFFFFFFFFFFFFFFFFFFD2
:10102E00FFFFFFFFFFFFFFFFFFFFFFFF00FFFF3F81
:10103E00CFF3FCFFFF00FCFCFCFCC33FFFFFFFFFF8
:10104E00FFFFFFFFFFFFFFFF00F3CC3FFFFFFFFFA0
:10105E00FF00FFFFFFFFFF00FFFFFFFFFFFFFFFF90
:10106E00FFFFFFFFC0FFFFFFFCF3CFFFFFC0CFCF9F
:10107E00CFCFF0FFFFFFFFFFFFFFFFFFFFFFFFFFE1
:10108E00FFFFFFFFFFFFFFFFFFFFFFFFFFFFFFFF62
:10109E00FFFFFFFFFFFF000F3F3FFFFFFFFFFFFFC1
:1010AE00FFFFFFFFFFFFFFFFFFFFFFFFFFFF3F3FC2
:1010BE000F0000F0FCFCFFFFFFFFFFFFFFFFFFFF35
:1010CE00FFFFFFFFFFFFFFFFFFFFFCFCF000FFFF36
:1010DE00FFFFFFFFFFFFFFFFFFFFFFFFFFFFFFFF12
:1010EE00FFFFFFFFFFFFFFFFFFFFFFFFFFFFFFFF02
:1010FE00CFCF03030000CFCFCFCFCFCFCFCF3FFF88
:10110E00FFFFFFFFFFFFFFFFFFFFFFFFFFFFFFFFE1
:10111E00FCFCFFFFFFFFFFFFFFFFFF00FFFFFFFFD6
:10112E00FFFFFFFFFFFFFFFFF3F3F3F3F3F3F3F321
:10113E00F3F3F3F3F3F3FCFFFFFFFFFFFFFFFFFFFC
:10114E00FFFFFFFFFFFFFFFFFFFFFFFFFFFFFFFFA1
:10115E00FFFFFFFFFFFFFFFFFFFF000F3F3FFFFF00
:10116E00FFFFFFFFFFFFFFFFFFFFFFFFFFFFFFFF81
:10117E00FFFF3F3F0F0000F00C0C030303030303BC
:10118E0003030303030303030303030303030C0C0F
:10119E00F000FF0000000000000000000000000052
:1011AE0000000000000000000000000000FFFF0033
:1011BE0000000000FF0000C0300C030000FF03031E
:1011CE0003030CF00000000000FFFF000000000011
:1011DE00FF0C33C00000000000FF303030300C0335
:1011EE000000000000FFFF00000000003F000000B4
:1011FE00030C3000003F0000000000000000000063
:10120E0000FFFF00000000000000000000000000D2
:10121E0000000000000000000000000000FF000FB2
:10122E003030C0C0C0C0C0C0C0C0C0C0C0C0C0C0D0
:10123E00C0C0C0C0C0C030300F0000F00C0C0303A3
:10124E000303030303030303030303030303030360
:10125E0003030C0CF000FF00000000000000000073
:10126E000000000000000000000000000000000070
:10127E0000FFFF0000000000FF0000C0300C030064
:10128E0000030303FF0303030000000000FFFF0041
:10129E0000000000FF0C33C0000000000000000042
:1012AE00FF0000000000000000FFFF000000000033
:1012BE003F000000030C3000003030303F30303043
:1012CE000000000000FFFF00000000000000000012
:1012DE000000000000000000000000000000000000
:1012EE0000FF000F3030C0C0C0C0C0C0C0C0C0C002
:1012FE00C0C0C0C0C0C0C0C0C0C030300F0000F001
:10130E000C0C03030303030303030303030303038D
:10131E000303030303030C0CF000FF0000000000A6
:10132E0000000000000000000000000000000000AF
:10133E000000000000FFFF0000000000FF0000C0E2
:10134E00300C030000FF030303033CF00000000019
:10135E0000FFFF0000000000FF0C33C00000000083
:10136E0000FF0000000000FF0000000000FFFF0073
:10137E00000000003F000000030C3000003F303042
:10138E00303C0F000000000000FFFF0000000000D6
:10139E00000000000000000000000000000000003F
:1013AE000000000000FF000F3030C0C0C0C0C0C041
:1013BE00C0C0C0C0C0C0C0C0C0C0C0C0C0C030303F
:1013CE000F0000F0FCFCFFFFFFFFFFFFFFFFFFFF22
:1013DE00FFFFFFFFFFFFFFFFFFFFFCFCF000FFFF23
:1013EE00FFFFFFFFFFFFFFFFFFFFFFFFFFFFFFFFFF
:1013FE00FFFFFFFFFFFFFFFFFFFFFFFFFFF30303F3
:10140E00FF0303F3FFFFFF3FC33FFFFFFFF3C333B2
:10141E00FF33C3F3FFFFFFFFFFFF00F00FF000FFEE
:10142E00FFFF3F003F003FFFFFFFFF3CC33CFFFFBE
:10143E00FFFFFFFFFFCFC0FFC0FFC0CFFFCFC0CF6A
:10144E00FFCFC0CFFFCFC3CCFFCCC3CFFFFFFFFF7B
:10145E00FFFFFFFFFFFFFFFFFFFFFFFFFFFFFFFF8E
:10146E00FFFFFFFFFFFFFFFFFFFF000F3F3FFFFFED
:10147E00FFFFFFFFFFFFFFFFFFFFFFFFFFFFFFFF6E
:10148E00FFFF3F3F0F0000F0FCFCFFFFFFFFFFFFE1
:10149E00FFFFFFFFFFFFFFFFFFFFFFFFFFFFFCFC54
:1014AE00F000FFFFFFFFFFFFFFFFFFFFFFFFFFFF4C
:1014BE00FFFFFFFFFFFFFFFFFFFFFFFFFFFFFFFF2E
:1014CE00FFF30303FF0303F3FFFFF3F303F3F3FF52
:1014DE00FFF30303FFF303F3FFFFFFFFFFFF00F034
:1014EE000FF000FFFFFFFFFF00FFFFFFFFFF00FFFA
:1014FE00C03F00FFFFFFFFFFFFCFC0FFC0FFC0CF09
:10150E00FFFFCFCFC0CFCFFFFFCFC0CFFFF0C0FFC9
:10151E00FFFFFFFFFFFFFFFFFFFFFFFFFFFFFFFFCD
:10152E00FFFFFFFFFFFFFFFFFFFFFFFFFFFF000FAC
:10153E003F3FFFFFFFFFFFFFFFFFFFFFFFFFFFFF2D
:10154E00FFFFFFFFFFFF3F3F0F0000F0FCFCFFFF20
:10155E00FFFFFFFFFFFFFFFFFFFFFFFFFFFFFFFF8D
:10156E00FFFFFCFCF000FFFFFFFFFFFFFFFFFFFF91
:10157E00FFFFFFFFFFFFFFFFFFFFFFFFFFFFFFFF6D
:10158E00FFFFFFFFFFFFFFFFCFCF03030000CFCF13
:10159E00CFCFCFCFCFCF3FFFFFFFFFFFFFFFFFFF2D
:1015AE00FFFFFFFFFFFFFFFFFCFCFFFFFFFFFFFF43
:1015BE00FFFFFF00FFFFFFFFFFFFFFFFFFFFFFFF2C
:1015CE00F3F3F3F3F3F3F3F3F3F3F3F3F3F3FCFFC8
:1015DE00FFFFFFFFFFFFFFFFFFFFFFFFFFFFFFFF0D
:1015EE00FFFFFFFFFFFFFFFFFFFFFFFFFFFFFFFFFD
:1015FE00FFFF000F3F3FFFFFFFFFFFFFFFFFFFFF5C
:10160E00FFFFFFFFFFFFFFFFFFFF3F3F0F0000F059
:10161E000C0C03030303030303030303030303037A
:10162E000303030303030C0CF000FF000000000093
:10163E00000000000000000000000000000000009C
:10164E000000000000FFFF00000CFCFC00FCFC0C86
:10165E00000000C03CC00000000C3CCC00CC3C0C98
:10166E0000FFFF000000FF0FF00FFF000000C0FFA3
:10167E00C0FFC000000000C33CC3000000FFFF001D
:10168E0000303F003F003F3000303F3000303F30F1
:10169E0000303C3300333C3000FFFF000000000000
:1016AE00000000000000000000000000000000002C
:1016BE000000000000FF000F3030C0C0C0C0C0C02E
:1016CE00C0C0C0C0C0C0C0C0C0C0C0C0C0C030302C
:1016DE000F0000F00C0C03030303030303030303C7
:1016EE00030303030303030303030C0CF000FF00C7
:1016FE0000000000000000000000000000000000DC
:10170E00000000000000000000FFFF00000CFCFCC9
:10171E0000FCFC0C00000C0CFC0C0C00000CFCFC87
:10172E00000CFC0C00FFFF000000FF0FF00FFF008D
:10173E0000000000FF0000000000FF003FC0FF009F
:10174E0000FFFF0000303F003F003F300000303010
:10175E003F30300000303F30000F3F0000FFFF00F1
:10176E00000000000000000000000000000000006B
:10177E00000000000000000000FF000F3030C0C06D
:10178E00C0C0C0C0C0C0C0C0C0C0C0C0C0C0C0C04B
:10179E00C0C030300F0000F00000000000FC000060
:1017AE00000000000000C03C0030F030303000007F
:1017BE00FC0030303030F0300C0C0C0C00000030DF
:1017CE00C000FC00C0300000FC00000000FF303004
:1017DE00303000FFC0300C030000300CFF0000F072
:1017EE000F0CFC00FF00FF0000303C33F030300CDB
:1017FE00C300000000C3330FFF0F33C3C03CC3034D
:10180E00FF0300FF0000C00000FF0000000000000A
:10181E000000FF000C030CF00F003F00FF000C0C4B
:10182E00CF0F0CFC0C0CCC0F3C00000CCCFF0C0CA6
:10183E00FC0000003FC03F00003F0C030000000F03
:10184E00303030303F0000003F00300C030000000D
:10185E0030303F000C030030303F000000030C001E
:10186E000030300C0F030C3000300C030C30C0C0B5
:10187E00C0303000F030303030F00000000000C0DA
:10188E003C0000003CC00000000030303030F03032
:10189E000C0C0C0C00000030C000FC00C03000002E
:1018AE00FC0000003030FF303000FF00000000FF71
:1018BE000000C030CCC3C0C0C0C0C0C30C30C0001C
:1018CE0000303C33F030300CC300000000C3330F47
:1018DE00FF0F33C3C03CC303FF03C03CFF030C0028
:1018EE0003C30303C3030000000000C03F00000059
:1018FE0000FF000000000C0CCF0F0CFC0C0CCC0FEA
:10190E003C00000CCCFF0C0CFC0000003FC03F0064
:10191E0000003F0000300C03000000033C00300CC0
:10192E00030000000030300F000000000C030030F8
:10193E00303F000000030C000030300C0F030C3061
:10194E0000300C030C3000C03CF000FC00F000FC3A
:10195E0000000000000000C03C0000003CC0000081
:10196E00000030303030F0300C0C0C0C0000003029
:10197E00C000FC00C0300000FC00000003C03CC3EF
:10198E00C3C3C3C30CF303FF0300C030CCC3C0C03A
:10199E00C0C0C0C30C30C00000303C33F030300C3F
:1019AE00C300000000C3330FFF0F33C3C03CC3039B
:1019BE00FF0303FF0000FC0CFC00000FF00F000003
:1019CE00000000C03F00000000FF000000000C0CF3
:1019DE00CF0F0CFC0C0CCC0F3C00000CCCFF0C0CF5
:1019EE00FC0000003FC03F00003F00300F000F031F
:1019FE00300F000F3000300C030000000030300FAD
:101A0E00000000000C030030303F000000030C000B
:101A1E000030300C0F030C3000300C030C30000083
:101A2E000CF00000F03030300C0C0C0C00000000FC
:101A3E0000FC0C0C0C0C0C0C0C0C0CFC0000000034
:101A4E000000000000000000000000000000000088
:101A5E0000000000303030F00000FF0CCC0C0C0CFD
:101A6E00CC3C0000000000FF0000FF030303FF005A
:101A7E0000FF000000000000000000000000000059
:101A8E0000000000000000000000000000FF00C089
:101A9E003F00C0330C33C0000000000000FF000008
:101AAE003F3030303F0000FF00000000000000001B
:101ABE000000000000000000000000000000000018
:101ACE0000300C030C3330333030303030333000D4
:101ADE000000003F0C0C0C0C0C0C0C0C0C3F00000E
:101AEE0000000000000000000000000000000000E8
:101AFE000000000000000000FCCCCCCCCCCCCCCC48
:101B0E00FC000000C0C0C0C0C0CCF0C0C0C0C0C08F
:101B1E00C00030C00000FC0C0C0C0CFC00000000DF
:101B2E0000C0C0C0C0CCF0C0C0C0C0C0C0C0CFCC10
:101B3E00CCCCCCCCCCCCCFC0C000000000FCCCCCEC
:101B4E00CCCCCCFC0000000C30000000FFC3C3C3A3
:101B5E00C3FF0000000000FF0C0CFFCCCCCCCCFF70
:101B6E000C0C00FFCCCCCCFF003CCC0CCC3C0000D1
:101B7E0000FC0C0CCCCCCCCCCC0C0CFC0000F00F34
:101B8E0000FC0CFC0C0CFC0CFC00000000FF000C1C
:101B9E003CCC0C0CCC3C0C000C0F0C0C033F03305B
:101BAE000C030C303000003F00000F0C0C0C0F002B
:101BBE00303F000F0000303F303F30303F303F307D
:101BCE0000300F0030300C0C03030C0C30300000D2
:101BDE00FCCCCCCCCCCCCCCCFC0000000000FC006F
:101BEE00C0C0C0C0F0303000000030C00000FC0C9F
:101BFE000C0C0CFC0000000000C0C0C0C0CCF0C03B
:101C0E00C0C0C0C0C0C0CFCCCCCCCCCCCCCCCFC054
:101C1E00C00030FF0000FFC0C0C0FFC0C0C0000C3D
:101C2E0030000000FFC3C3C3C3FF0000000000FF6D
:101C3E000C0CFFCCCCCCCCFF0C0C00FFCCCCCCFFD6
:101C4E00003CCC0CCC3C000000FF0000FF00C000AC
:101C5E003FC000000000F00F00FC0CFC0C0CFC0C54
:101C6E00FC00000000FF000C3CCC0C0CCC3C0C002B
:101C7E000C0F0C0C033F03300C030C303000003FF4
:101C8E0000000F03000C30030C3F000F0000303F2C
:101C9E00303F30303F303F3000300F0030300C0CD2
:101CAE0003030C0C303000000CF00000F03030302C
:101CBE000C0C0C0C0000000000FC0C0C0C0C0C0CA2
:101CCE000C0C0CFC000000000000000000000000E6
:101CDE00000000000000000000000000303030F076
:101CEE000000FF0CCC0C0C0CCC3C0000000000FFE4
:101CFE000000FF030303FF0000FF000000000000D0
:101D0E0000000000000000000000000000000000C5
:101D1E000000000000FF00C03F00C0330C33C000C5
:101D2E000000000000FF00003F3030303F0000FF99
:101D3E000000000000000000000000000000000095
:101D4E00000000000000000000300C030C333033A4
:101D5E0030303030303330000000003F0C0C0C0CB3
:101D6E000C0C0C0C0C3F00000000000000000000EA
:101D7E00000000000000000000000000000000F065
:101D8E00FCFCFFFFFFFFFFFFFFFFFFFFFFFFFFFF5B
:101D9E00FFFFFFFFFFFFFCFCF000FFFFFFFF003C1B
:101DAE003C00FFFF3C3C3C3C3C3C3C3C3C3C3C3C1B
:101DBE003C3CFFFFFFFFFFFFFFFFFFFFFFFFFFFFAB
:101DCE00FFFFFFFFFFFFFFFFFFFFFFFFFFFFFFFF15
:101DDE00FFFFFFFFFFFF003C3C00FFFF3C3C3C3C95
:101DEE003C3C3C3C3C3C3C3C3C3CFFFFFFFFFFFF93
:101DFE00FFFFFFFFFFFFFFFFFFFFFFFFFFFFFFFFE5
:101E0E00FFFFFFFFFFFFFFFFFFFFFFFFFFFF003C96
:101E1E003C00FFFF3C3C3C3C3C3C3C3C3C3C3C3CAA
:101E2E003C3CFFFFFFFF000F3F3FFFFFFFFFFFFFA9
:101E3E00FFFFFFFFFFFFFFFFFFFFFFFFFFFF3F3F24
:101E4E000F0000F0FCFCFFFFFFFFFFFFFFFFFFFF97
:101E5E00FFFFFFFFFFFFFFFFFFFFFCFCF000FFFF98
:101E6E00FFFF00FFFFFFFFFFFFFFFFFFFFFFFFFF73
:101E7E00FFFFFFFFFFFFFFFFFFFFFFFFFFFF00FF63
:101E8E00FFFFFF0FF3FCFCFCF3CF3FFFFFFFFFFF55
:101E9E00FFFFFFFFFFFFFFFFFFFF00FFFF0FF0FF42
:101EAE00FFFFFFFFFFFFFFFCF3F3F3F3F3F3FFFF7F
:101EBE00FFFFFFFFFFFF00FF03FCFFFFFFFFFFFF22
:101ECE00FFFFFFFFFFFFFFFFFFFFFFFFFFFFFFFF14
:101EDE00FFFF00003F3F3F3F3F3F3F3F3F3F3F3F02
:101EEE003F3F3F3F3F3FFFFFFFFF000F3F3FFFFFE3
:101EFE00FFFFFFFFFFFFFFFFFFFFFFFFFFFFFFFFE4
:101F0E00FFFF3F3F0F0000F0FCFCFFFFFFFFFFFF56
:101F1E00FFFFFFFFFFFFFFFFFFFFFFFFFFFFFCFCC9
:101F2E00F000FFFFFFFFFFFFFFFFFFFFFFFFFFFFC1
:101F3E00FFFFFFFFFFFFFFFFFFFFFFFFFFFFFFFFA3
:101F4E00FFFFFFFFCFCF03030000CFCFCFCFCFCF09
:101F5E00CFCF3FFFFFFFFFFFFFFFFFFFFFFFFFFFA3
:101F6E00FFFFFFFFFCFCFFFFFFFFFFFFFFFFFF0078
:101F7E00FFFFFFFFFFFFFFFFFFFFFFFFF3F3F3F393
:101F8E00F3F3F3F3F3F3F3F3F3F3FCFFFFFFFFFFCE
:101F9E00FFFFFFFFFFFFFFFFFFFFFFFFFFFFFFFF43
:101FAE00FFFFFFFFFFFFFFFFFFFFFFFFFFFF000F22
:101FBE003F3FFFFFFFFFFFFFFFFFFFFFFFFFFFFFA3
:101FCE00FFFFFFFFFFFF3F3F0F0000F00C0C03036E
:101FDE0003030303030303030303030303030303C3
:101FEE0003030C0CF000FF000000FFC3C3FF000052
:101FFE00C3C3C3C3C3C3C3C3C3C3C3C3C3C3000029
:10200E0000FFFF00000000000000000000000000C4
:10201E0000000000000000000000000000FFFF00B4
:10202E000000FFC3C3FF0000C3C3C3C3C3C3C3C306
:10203E00C3C3C3C3C3C3000000FFFF000000000002
:10204E000000000000000000000000000000000082
:10205E000000000000FFFF000000FFC3C3FF0000F0
:10206E00C3C3C3C3C3C3C3C3C3C3C3C3C3C30000B8
:10207E0000FF000F3030C0C0C0C0C0C0C0C0C0C064
:10208E00C0C0C0C0C0C0C0C0C0C030300F0000F063
:10209E000C0C0303030303030303030303030303F0
:1020AE000303030303030C0CF000FF000000FF000A
:1020BE000000000000000000000000000000000012
:1020CE000000000000FFFF000000FF00000000F015
:1020DE000C0303030C30C0000000000000000000E1
:1020EE0000FFFF000000FF0000F00F0000000000E6
:1020FE00000000030C0C0C0C0C0C000000FFFF0089
:10210E000000FF00FC0300000000000000000000C3
:10211E00000000000000000000FFFF000000FFFFB5
:10212E00C0C0C0C0C0C0C0C0C0C0C0C0C0C0C0C0A1
:10213E00C0C0000000FF000F3030C0C0C0C0C0C023
:10214E00C0C0C0C0C0C0C0C0C0C0C0C0C0C03030A1
:10215E000F00000CF000000C30000000300C0000EE
:10216E0000C03C00C000F03030F03030F000000015
:10217E00C03CC0C0C0CCF0C0C0C0C00000C0C0F0E9
:10218E00CCC0C0C0C0C000003030F00000C3C3C31C
:10219E00FFC3C3C300000C0FCC3C0300FFC0C0FF45
:1021AE00C0C0FF00300CFF0000CCCCCCCCCCCCCCD3
:1021BE00000000FFCCCCCCCCCCCCCCFF000000007F
:1021CE00FF0030303030FF30303030000C0F0C0C50
:1021DE000C00FF0000FF0000FF000000FF0000FCED
:1021EE000C0C0C0C0CFC0000000FCC0C0C3CCC0CA2
:1021FE000C0FC00000000F03000000003F000000A5
:10220E0000000C0C0C0303003F0C0C0F0C0C3F00D9
:10221E0000003F00003F0C0C0C0C0C3F00300F0078
:10222E000F30303033303C00000F0030C00000FC67
:10223E000C0C0C0CFC0000000000C0C0C0C0CCF0A8
:10224E00C0C0C0C0C00000000000FC0000FC0000C8
:10225E0000000000C03C00C0000000FC000C30007C
:10226E000C30000000FFC3C3C3C3FF00000000001A
:10227E00FF0C0CFFCCCCCCCCFF0C0C00FF030303EB
:10228E00FF0303FF030303FF000C0FCC3C03000C02
:10229E000CFF03C3C3C000F00F00FC0CFC0C0CFCC5
:1022AE000CFC00000000FF000C3CCC0C0CCC3C0CD9
:1022BE000000FF030303FF0303FF030303FF000CF0
:1022CE000F0C0C0C0003033FC3300CC00F0000308A
:1022DE003F303F30303F303F3000300F0030300C59
:1022EE000C03030C0C3030003F0C0C0C0F0C0C0FBD
:1022FE000C0C0C3F000C0C0C0303000C0C03000325
:10230E000C3F00000CF00000F03030300C0C0C0CC8
:10231E000000000000FC0C0C0C0C0C0C0C0C0CFC4B
:10232E00000000000000000000000000000000009F
:10233E000000000000000000303030F00000FF0C04
:10234E00CC0C0C0CCC3C0000000000FF0000FF0386
:10235E000303FF0000FF000000000000000000006B
:10236E00000000000000000000000000000000005F
:10237E0000FF00C03F00C0330C33C000000000005F
:10238E0000FF00003F3030303F0000FF0000000033
:10239E00000000000000000000000000000000002F
:1023AE000000000000300C030C333033303030307E
:1023BE00303330000000003F0C0C0C0C0C0C0C0CDD
:1023CE000C3F0000000000000000000000000000B4
:1023DE0000000000000000000000F0FCFFFFFFFF07
:1023EE00FFFFFF0F030303030CF01F7FFFFFFFFF31
:1023FE00FFFFFFE080808080601FF00CC3F3F3C30B
:10240E0003030303030303030CF00F30C3CFCFC347
:10241E00C0C0C0C0C0C0C0C0300F3F000000000030
:10242E00000000000000000000000000000000009E
:10243E00000000000000000000000000000000008E
:10244E00000000000000000000000000000000007E
:10245E00000000000000000000000000000000006E
:10246E00000000000000000000000000000000005E
:10247E00000000000000000000000000000000004E
:10248E00003F0000000000000000000000000000FF
:10249E00000000000000000000000000000000002E
:1024AE00000000000000000000000000000000001E
:1024BE00000000000000000000000000000000000E
:1024CE0000000000000000000000000000000000FE
:1024DE0000000000000000000000000000000000EE
:1024EE0000000000000000003F000000000000009F
:1024FE0000000000000000000000000000000000CE
:10250E0000000000000000000000000000000000BD
:10251E0000000000000000000000000000000000AD
:10252E00000000000000000000000000000000009D
:10253E00000000000000000000000000000000008D
:10254E000000000000000000000000000000003F3E
:10255E00000000000000000000000000000000006D
:10256E00000000000000000000000000000000005D
:10257E00000000000000000000000000000000004D
:10258E00000000000000000000000000000000003D
:10259E00000000000000000000000000000000002D
:1025AE00000000000000000000000000000000001D
:1025BE000000000000003F000000000000000000CE
:1025CE0000000000000000000000000000000000FD
:1025DE0000000000000000000000000000000000ED
:1025EE0000000000000000000000000000000000DD
:1025FE0000000000000000000000000000000000CD
:10260E0000000000000000000000000000000000BC
:10261E00000000000000000000000000003F00006D
:10262E00000000000000000000000000000000009C
:10263E00000000000000000000000000000000008C
:10264E00000000000000000000000000000000007C
:10265E00000000000000000000000000000000006C
:10266E00000000000000000000000000000000005C
:10267E00000000000000000000000000000000004C
:10268E00000000003F0000000000000000000000FD
:10269E00000000000000000000000000000000002C
:1026AE00000000000000000000000000000000001C
:1026BE00000000000000000000000000000000000C
:1026CE0000000000000000000000000000000000FC
:1026DE0000000000000000000000000000000000EC
:1026EE000000000000000000000000FFC0C0C0C0DD
:1026FE00C0C0C000C0C0C0C0C0C0C000C0C0C0C04C
:10270E00C0C0C000C0C0C0C0C0C0C000C0C0C0C03B
:10271E00C0C0C000C0C0C0C0C0C0C000C0C0C0C02B
:10272E00C0C0C000C0C0C0C0C0C0C000C0C0C0C01B
:10273E00C0C0C000C0C0C0C0C0C0C000C0C0C0C00B
:10274E00C0C0C000C0C0C0C0C0C0C000C0C0C0C0FB
:02275E00C0C0F9
:1041A7004204BF01F4420408012C4204C10000424A
:1041B70004C300004204A200004204B8015E4204A6
:1041C700B600014204BC000A4204B200144204B023
:1041D700001E4204B400004205AB00004204AA00DE
:1041E7000042040200004204BA00004204A4000096
:1041F70044040C000000004404AC00000000607898
:10420700052E000000000000000000000000000074
:104217000000000000000000000000000000000097
:104227000000000000000000000000000000000087
:104237000000000000000000000000000000000077
:104247000000000000000000000000000000000067
:104257000000000000000000000000000000000057
:104267000000000000000000000000000000000047
:10427700000000000000000000004405A7434800BC
:104287000060780428000000000000000000000023
:104297000000000000000000000000000000000017
:1042A7000000000000000000000000000000000007
:1042B70000000000000000000000000000000000F7
:1042C70000000000000000000000000000000000E7
:1042D70000000000000000000000000000000000D7
:1042E70000000000000000000000000000000000C7
:1042F700000000000000000000000000004404115E
:10430700342BCC77440415BA6A76D74404193FF4A2
:10431700F36C44041DC4C03F304404A600000000F1
:1043270041042600410410004105A600410427046A
:104337004104BE0441052C03410421034205B30097
:104347000042040A00004204060000420404000080
:104357004205B100004205AF0000606504C70000D8
:104367000000000000000000000000000000000046
:104377000000000000000000000000000000000036
:104387000000000000000000000000000000000026
:104397000000000000000000000000000000000016
:1043A7000000000000000000000000000000000006
:1043B70000000000000000000000000000000000F6
:1043C70000000041052D1EC180C18BC182C18AC179
:0143D7008164
:086F9F009005B5EFF0A3EDF041
:106FA7007C007D0AAF03AE02125197A3EDF07C007F
:106FB7007D0AAF03AE021251977C007D0A125197EA
:106FC700A3EDF0AE02AF037C007D641251977C0005
:106FD7007D0A125197AF05EF75F060A4240EF9747E
:106FE7000035F0FA9005C474FFF0A3EAF0A3E9F0C6
:106FF7009005B5E0FFA3E0FD9005C37430F07B106A
:10700700126DB69005B5E02410F09005B8E075F064
:1070170060A4240EF9740035F0FA9005C474FFF0EB
:10702700A3EAF0A3E9F09005B5E0FFA3E0FD900522
:10703700C37430F07B10126DB69005B5E02410F0E4
:107047009005B7E075F060A4240EF9740035F0FAE6
:107057009005C474FFF0A3EAF0A3E9F09005B5E04A
:0F706700FFA3E0FD9005C37430F07B10026DB6FF
:086CBC009005B5EFF0A3EDF027
:106CC4007C007D0AAF03AE021251979005BAEDF035
:106CD4007C007D0AAF03AE021251977C007D0A123C
:106CE4005197A3EDF0AE02AF037C007D641251977F
:106CF400EF75F018A424CEF9740335F0FA9005C4A6
:106D040074FFF0A3EAF0A3E9F09005B5E0FFA3E077
:106D1400FD9005C37418F07B08126DB69005B5E0BC
:106D24002408F09005BBE075F018A424CEF9740390
:106D340035F0FA9005C474FFF0A3EAF0A3E9F090EB
:106D440005B5E0FFA3E0FD9005C37418F07B0812BD
:106D54006DB69005B5E02408F09005BAE075F0181A
:106D6400A424CEF9740335F0FA9005C474FFF0A39B
:106D7400EAF0A3E9F09005B5E0FFA3E0FD9005C3B8
:106D84007418F07B08126DB69005B9E06023900585
:106D9400B5E02408F0E0FFA3E0FD9005C37418F00B
:106DA400A374FFF0A37405F0A37403F07B0B126DBE
:016DB400B628
:016DB50022BB
:085BCA009005B5EFF0A3EDF02A
:105BD200E4FFFE7D207C41A3E0F8A3E0F9A3E0FA14
:105BE200A3E0FB124FF54003025D31E4FFFE7DC8E6
:105BF2007C429005B7E0F8A3E0F9A3E0FAA3E0FB4A
:105C0200124E4F1250AC9005BEEEF0A3EFF090058D
:105C1200BEE0FAA3E0FB7C007D64FFAE0212519766
:105C22009005BBEFF07C007D0AAF03AE02125197E4
:105C32007C007D0A125197A3EDF09005BEE0FEA311
:105C4200E0FF7C007D0A1251979005BDEDF09005B2
:105C5200BBE075F018A424CEF9740335F0FA900570
:105C6200C474FFF0A3EAF0A3E9F09005B5E0FFA346
:105C7200E0FD9005C37418F07B08126DB69005B56F
:105C8200E02408F0E0FFA3E0FD9005C37418F0A340
:105C920074FFF0A37405F0A3743CF07B02126DB69E
:105CA2009005B5E02402F09005BCE075F018A4243C
:105CB200CEF9740335F0FA9005C474FFF0A3EAF04C
:105CC200A3E9F09005B5E0FFA3E0FD9005C37418C9
:105CD200F07B08126DB69005B5E02408F09005BD82
:105CE200E075F018A424CEF9740335F0FA9005C4D7
:105CF20074FFF0A3EAF0A3E9F09005B5E0FFA3E09A
:105D0200FD9005C37418F07B08126DB69005B5E0DE
:105D12002408F0E0FFA3E0FD9005C37418F0A3741B
:105D2200FFF0A37405F0A37424F07B08126DB6E4AF
:105D3200FFFE7D207C419005B7E0F8A3E0F9A3E0E7
:105D4200FAA3E0FB124FF55003025E92E4FFFE7DE0
:105D5200207C419005B7E0F8A3E0F9A3E0FAA3E0C4
:105D6200FB124E4F1250AC9005BEEEF0A3EFF09036
:105D720005BEE0FAA3E0FB7C007D64FFAE02125197
:105D8200979005BBEFF07C007D0AAF03AE02125183
:105D9200977C007D0A125197A3EDF09005BEE0FEBC
:105DA200A3E0FF7C007D0A1251979005BDEDF090B3
:105DB20005BBE075F018A424CEF9740335F0FA900F
:105DC20005C474FFF0A3EAF0A3E9F09005B5E0FF83
:105DD200A3E0FD9005C37418F07B08126DB6900520
:105DE200B5E02408F09005BCE075F018A424CEF9C3
:105DF200740335F0FA9005C474FFF0A3EAF0A3E946
:105E0200F09005B5E0FFA3E0FD9005C37418F07BA8
:105E120008126DB69005B5E02408F0E0FFA3E0FD9E
:105E22009005C37418F0A374FFF0A37405F0A37473
:105E32003CF07B02126DB69005B5E02402F09005AD
:105E4200BDE075F018A424CEF9740335F0FA90057C
:105E5200C474FFF0A3EAF0A3E9F09005B5E0FFA354
:105E6200E0FD9005C37418F07B08126DB69005B57D
:105E7200E02408F0E0FFA3E0FD9005C37418F0A34E
:105E820074FFF0A37405F0A37424F07B08126DB6BE
:015E920022ED
:0B6944009005B5EFF0A3EDF0A3EBF021
:10694F00A3E0601075F035A4FFAEF07C007D6412FB
:10695F005197EFF09005B5E0FFA3E0FD9005C374EC
:10696F0010F0A374FFF0A37405F0A37442F07B370B
:10697F00126DB69005B7E0146074046003026A7E6E
:10698F009005B6E0FD9005C37410F0A374FFF0A35B
:10699F007405F0A374B0F07B08E4FF126DB6900598
:1069AF00B8E07003026A7EE4A3F09005B8E014FF2C
:1069BF00A3E0FEC39F50289005B5E02E04FBFFA374
:1069CF00E075F008A4FE2402FDEE240D9005BFF043
:1069DF00A37401F01256129005B9E004F080CB9029
:1069EF0005B8E0FF9005B5E02FFBFFA3806A900587
:1069FF00B6E0FD9005C37410F0A374FFF0A3740507
:106A0F00F0A374C0F07B087F78126DB69005B8E0E4
:106A1F00605DE4A3F09005B8E014FFA3E0FEC39F10
:106A2F005028C374769EFBFF9005B6E075F008A45E
:106A3F00FE2402FDEE240D9005BFF0A37401F012A9
:106A4F0056129005B9E004F080CB9005B8E0FFC373
:106A5F0074779FFBFF9005B6E075F008A4FE240441
:0F6A6F00FDEE240B9005BFF0A37401F012561238
:016A7E0022F5
:105E93009005B5EFF0A3EDF0A3EBF06011E075F022
:105EA30030A4FFAEF07C007D64125197EFF09005B3
:105EB300BAE0FEA3E0FFD39005B9E09F9005B8E0F8
:105EC3009E9005B7E0FF9005B5E05003025FCD2F2C
:105ED30024FEFBFFA3E0FE2406FDEE24099005BF8C
:105EE300F0A37401F01256129005B7E0FF9005B5C8
:105EF300E02F14FBFFA3E0FE2404FDEE240B90052A
:105F0300BFF0A37401F01256129005B7E0FF90059D
:105F1300B5E02F14FBFFA3E0FE2406FDEE24099059
:105F230005BFF0E4A3F01256129005B7E0FF900509
:105F3300B5E02FFBFFA3E0FE2402FDEE240D900548
:105F4300BFF0A37401F01256129005B7E0FF90055D
:105F5300B5E02FFBFFA3E0FE2404FDEE240B900528
:105F6300BFF0E4A3F01256129005B7E0FF9005B519
:105F7300E02F04FBFFA3E0FE2404FDEE240B9005B9
:105F8300BFF0A37401F01256129005B7E0FF90051D
:105F9300B5E02F04FBFFA3E0FE2406FDEE240990E9
:105FA30005BFF0E4A3F01256129005B7E0FF900589
:105FB300B5E02F2402FBFFA3E0FE2406FDEE240937
:105FC3009005BFF0A374010260C32F24FEFBFFA35F
:105FD300E0FE2406FDEE24099005BFF0E4A3F012D1
:105FE30056129005B7E0FF9005B5E02F14FBFFA311
:105FF300E0FE2404FDEE240B9005BFF0E4A3F012B1
:1060030056129005B7E0FF9005B5E02F14FBFFA3F0
:10601300E0FE2406FDEE24099005BFF0A37401F011
:106023001256129005B7E0FF9005B5E02FFBFFA3D2
:10603300E0FE2402FDEE240D9005BFF0E4A3F01270
:1060430056129005B7E0FF9005B5E02FFBFFA3E0E4
:10605300FE2404FDEE240B9005BFF0A37401F0129F
:1060630056129005B7E0FF9005B5E02F04FBFFA3A0
:10607300E0FE2404FDEE240B9005BFF0E4A3F01230
:1060830056129005B7E0FF9005B5E02F04FBFFA380
:10609300E0FE2406FDEE24099005BFF0A37401F091
:1060A3001256129005B7E0FF9005B5E02F2402FBCE
:1060B300FFA3E0FE2406FDEE24099005BFF0E4A350
:0560C300F0125612224C
:0E60C8009005B5EFF0A3EDF0A3EAF0A3EBF026
:1060D600A3E0640360030261919005B7E0FAA3E0D0
:1060E600FB7C007D64FFAE021251979005BAEFF07B
:1060F6007C007D0AAF03AE021251977C007D0A1226
:106106005197A3EDF09005B7E0FEA3E0FF7C007D7C
:106116000A1251979005BCEDF09005BAE075F0189B
:10612600A424CEF9740335F0FA9005C474FFF0A3E5
:10613600EAF0A3E9F09005B5E0FFA3E0FD9005C302
:106146007418F07B08126DB69005B5E02408F0903F
:1061560005BBE075F018A424CEF9740335F0FA9067
:1061660005C474FFF0A3EAF0A3E9F09005B5E0FFDB
:10617600A3E0FD9005C37418F07B08126DB6900578
:10618600B5E02408F09005BC0262969005B9E0647B
:106196000460030262C29005B7E0FAA3E0FB7C0349
:1061A6007DE8FFAE021251979005BAEFF07C007DB4
:1061B60064AF03AE021251977C007D0A125197A379
:1061C600EDF09005B7A3E07C007D0AFFAE02125108
:1061D600977C007D0A1251979005BCEDF07C007DFE
:1061E6000AAF03AE02125197A3EDF09005BAE0751F
:1061F600F018A424CEF9740335F0FA9005C474FFA0
:10620600F0A3EAF0A3E9F09005B5E0FFA3E0FD9066
:1062160005C37418F07B08126DB69005B5E0240826
:10622600F09005BBE075F018A424CEF9740335F0A0
:10623600FA9005C474FFF0A3EAF0A3E9F09005B55F
:10624600E0FFA3E0FD9005C37418F07B08126DB65D
:106256009005B5E02408F09005BCE075F018A4247C
:10626600CEF9740335F0FA9005C474FFF0A3EAF092
:10627600A3E9F09005B5E0FFA3E0FD9005C374180F
:10628600F07B08126DB69005B5E02408F09005BDC8
:10629600E075F018A424CEF9740335F0FA9005C41D
:1062A60074FFF0A3EAF0A3E9F09005B5E0FFA3E0E0
:0C62B600FD9005C37418F07B08126DB653
:0162C20022B9
:1047E1007B017A0579B39005BAE4F0A37402F0E491
:1047F100FFFE12776D7B017A04790A9005BAE4F025
:10480100A37402F07F00FE12776D7B017A047906B2
:104811009005BAE4F0A37402F07F04FE12776D7B79
:10482100017A0479049005BAE4F0A37402F07F08D8
:10483100FE12776D7B017A0579B19005BAE4F0A398
:104841007402F07F007E0412776D7B017A0579AFE7
:104851009005BAE4F0A37402F07404FFFE12776DC0
:104861007B017A0579A69005BAE4F0A304F07F00F4
:104871007E0612776D9005B4E0FE9005B3E07C00F2
:104881002400FFEC3E900408F0A3EFF090040BE04D
:10489100FE90040AE02400FFEC3E9004BCF0A3EF7C
:1048A100F0900407E0FE900406E02400FFEC3E9047
:1048B10004B2F0A3EFF0900405E0FE900404E024BC
:1048C10000FFEC3E9004B0F0A3EFF09005B2E0FEE3
:1048D1009005B1E02400FFEC3E9004B8F0FCA3EF9A
:1048E100F0FD9005B0E0FE9005AFE07A002400FFF6
:1048F100EA3E9004B6F0A3EFF0D3ED945EEC9401A0
:10490100400AA37401F0A3745EF08015C39004B94A
:10491100E094C89004B8E094005006E4F0A374C891
:10492100F09004B6E0FEA3E0D394C8EE94004002F8
:104931008006C3EE94005007E49004B6F0A3F09013
:1049410004B8E0FEA3E0FF900408E0FCA3E0FDD37F
:104951009FEC9E4002800F9004B6E0FEA3E0FFC3EF
:10496100ED9FEC9E5008900408EEF0A3EFF0900448
:10497100BCE0FEA3E0D394E8EE9403400C9004BCA9
:104981007401F0A374F4F0800DC3EE94005007E4B9
:104991009004BCF0A3F09004B2E0FEA3E0D394E84D
:1049A100EE9403400C9004B27401F0A374F4F0800F
:1049B1000DC3EE94005007E49004B2F0A3F090040C
:1049C100B0E0FEA3E0D394E8EE9403400C9004B071
:1049D1007401F0A374F4F0800DC3EE94005007E469
:1049E1009004B0F0A3F0900421E0FF24FEFE9005B6
:1049F100A6E0D39E5006EFC394005005E49005A6AF
:104A0100F0E4F5927591FF75B2FF75B10CC2B4C2B5
:104A1100009004221252680000000012799612746C
:104A210046127931D2AF90040CE0F8A3E0F9A3E08B
:104A3100FAA3E0FBE4FFFE7DC87C42124D5A9004CC
:104A4100AC12525CE49004C5F0A3F090052DE0FF98
:104A5100C39004C6E09F9004C5E094004003024B5C
:104A610043E4FFFE127394AC06AD07E4125073C029
:104A710004C005C006C0079004C5E0FEA3E07802AB
:104A8100C333CE33CED8F9242EF58274053EF58397
:104A9100D007D006D005D00412525C7F017E0012EF
:104AA1007394C006C007900411E0FCA3E0FDA3E0ED
:104AB100FEA3E0FF9005B712525C900415E0FCA341
:104AC100E0FDA3E0FEA3E0FF9005BB12525C900461
:104AD10019E0FCA3E0FDA3E0FEA3E0FF9005BF12F7
:104AE100525C90041DE0FCA3E0FDA3E0FEA3E0FF07
:104AF1009005C312525CD007D006126EADAC06AD64
:104B010007E4125073C004C005C006C0079004C575
:104B1100E0FEA3E07802C333CE33CED8F92428F5E2
:104B21008274043EF583D007D006D005D00412521A
:104B31005C9004C6E004F070069004C5E004F00245
:104B41004A4CE49004C5F0A3F090052DE0FFC3901A
:104B510004C6E09F9004C5E0940050599004A6E07B
:104B6100F8A3E0F9A3E0FAA3E0FBC000C001C00292
:104B7100C0037F0F7E00127394AC06AD07E41250A0
:104B810073A804A905AA06AB077FEC7E517D987C2A
:104B910045124F58D003D002D001D000124D5E9083
:104BA10004A612525C9004C6E004F0709C9004C507
:104BB100E004F080949004A6E0FCA3E0FDA3E0FEF5
:104BC100A3E0FFC004C005C006C00790052DE0FCAE
:104BD100E4125078A804A905AA06AB07D007D006AD
:104BE100D005D004124F589004A612525CE49004F0
:104BF100C5F0A3F090052DE0FFC39004C6E09F909F
:104C010004C5E094004003024CE7900422E0F8A3BD
:104C1100E0F9A3E0FAA3E0FBC000C001C002C003B9
:104C21009004C5E0FEA3E07802C333CE33CED8F9B9
:104C3100242EF58274053EF583E0FCA3E0FDA3E09C
:104C4100FEA3E0FFE4FBFA79807845124F58C004D7
:104C5100C005C006C007E4FFFE7D987C419004A614
:104C6100E0F8A3E0F9A3E0FAA3E0FB124E4FD00372
:104C7100D002D001D000124E4FD003D002D001D0CB
:104C810000124D5E90042212525C9005A7E0FCA335
:104C9100E0FDA3E0FEA3E0FFC004C005C006C0071D
:104CA1009004C5E0FEA3E07802C333CE33CED8F939
:104CB1002428F58274043EF583E0F8A3E0F9A3E02B
:104CC100FAA3E0FBD007D006D005D004124D5E90C8
:104CD10005A712525C9004C6E004F070069004C56A
:104CE100E004F0024BF5900422E0FCA3E0FDA3E018
:104CF100FEA3E0FFC004C005C006C00790052DE07B
:104D0100FCE4125078A804A905AA06AB07D007D085
:104D110006D005D004124F5890042212525C90051F
:104D2100A7E0FCA3E0FDA3E0FEA3E0FFC004C005F3
:104D3100C006C00790052DE0FCE4125078A804A934
:104D410005AA06AB07D007D006D005D004124F58EC
:064D51009005A702525C70
:107904001247E1900410E070031252C5900410E095
:08791400B401F012276080EBC2
:03000B000274F18B
:1074F100C0E0C0F0C083C082C0D075D000C000C061
:1075010001C002C003C004C005C006C0079004A1A9
:10751100E004F070069004A0E004F09004A0E0FE06
:10752100A3E0FF7C037DE81251979004A0ECF0FEEC
:10753100A3EDF0FF7C037DE8125197ED4C7007C27B
:1075410009300002D2069004A0E0FEA3E0FFC39040
:1075510004B5E09F9004B4E09E4007300004D2B42B
:107561008002C2B412760FD007D006D005D004D065
:1075710003D002D001D000D0D0D082D083D0F0D0BF
:02758100E032F6
:10760F0020B21630B3132003109004C2E004F070C0
:10761F00069004C1E004F0D20720B31630B2132055
:10762F0003109004C4E004F070069004C3E004F06B
:10763F00D20820B24320B3409004BFE0FEA3E0FF86
:10764F00C39004C2E09F9004C1E09E502BC39004EE
:10765F00C4E09F9004C3E09E501EC208C207E4F02E
:10766F00A3F09004C1F0A3F09004A3E004F070061F
:09767F009004A2E004F0D2032201
:1062C30020B2399004BFE0FEA3E0FFC39004C2E014
:1062D3009F9004C1E09E40249004B8E0FEA3E0FF39
:1062E300900409E09F900408E09E5042A3E004F06C
:1062F3007006900408E004F0C20B803230B22F30F5
:10630300072C9004B8E0FEA3E0FFC3900409E09FCC
:10631300900408E09E5017A3E004F0700690040870
:10632300E004F0E49004C1F0A3F0C207C20B20B371
:106333003A9004BFE0FEA3E0FFC39004C4E09F9043
:1063430004C3E09E40259004B6E0FEA3E0FFD39093
:106353000409E09F900408E09E4045A3E024FFF079
:10636300900408E034FFF0C20B803530B3323008BC
:106373002F20052C9004B6E0FEA3E0FFD390040980
:10638300E09F900408E09E4017A3E024FFF09004F0
:1063930008E034FFF0E49004C3F0A3F0C208C20B9A
:1063A30020B24720B3449004BFE0FEA3E0FFC390B4
:1063B30004A3E09F9004A2E09E402F30032C3004FE
:1063C30029900410E070047F0180027F0090041084
:1063D300EFF0C200C2B4C203E49004A2F0A3F0C27F
:1063E300049005ABF0A304F0804430B34130B23ED7
:1063F30030033B9004BFE0FEA3E0FFC39004A3E09F
:106403009F9004A2E09E5026300423B2009005AB77
:10641300E4F0A304F0A20092B4E49004BAF0A3F071
:106423009004B4F0A3F0C2039004A2F0A3F030B33D
:106433005330B250E49004A2F0A3F0C203D204900C
:1064430004C1F0A3F0A3F0A3F0C207C208200B34E9
:10645300900408E0FEA3E09005B3F0EEA3F0E4FFA0
:10646300FE1279447B017A0579B39005BAE4F0A36F
:106473007402F0E4FFFE127734E49005B4F0900563
:0A648300B3F0D20B300502C205226F
:1052C5001278D0900426E004F0E0FF90052DE0FE72
:1052D500EF8EF084900426E5F0F0E4FFFE1273945F
:1052E500AC06AD07E4125073900426E025E025E0F6
:1052F500242EF582E43405F58312525C7F017E008D
:10530500127394C006C007900411E0FCA3E0FDA34E
:10531500E0FEA3E0FF9005B712525C900415E0FC97
:10532500A3E0FDA3E0FEA3E0FF9005BB12525C9055
:105335000419E0FCA3E0FDA3E0FEA3E0FF9005BF98
:1053450012525C90041DE0FCA3E0FDA3E0FEA3E087
:10535500FF9005C312525CD007D006126EADAC06A5
:10536500AD07E4125073900426E025E025E02428DB
:10537500F582E43404F58312525C9005A712526855
:105385000000000090042212526800000000900402
:10539500A612526800000000E49004C5F0A3F09046
:1053A500052DE0FFC39004C6E09F9004C5E094007E
:1053B50050599004A6E0F8A3E0F9A3E0FAA3E0FBB6
:1053C500C000C001C002C0037F0F7E00127394AC01
:1053D50006AD07E4125073A804A905AA06AB077F1A
:1053E500EC7E517D987C45124F58D003D002D001F8
:1053F500D000124D5E9004A612525C9004C6E004E3
:10540500F070069004C5E004F080949004A6E0FCDA
:10541500A3E0FDA3E0FEA3E0FFC004C005C006C0F5
:105425000790052DE0FCE4125078A804A905AA060A
:10543500AB07D007D006D005D004124F589004A66C
:1054450012525CE49004C5F0A3F090052DE0FFC373
:105455009004C6E09F9004C5E094004003025541C6
:10546500900422E0F8A3E0F9A3E0FAA3E0FBC00072
:10547500C001C002C0039004C5E0FEA3E07802C3EA
:1054850033CE33CED8F9242EF58274053EF583E06C
:10549500FCA3E0FDA3E0FEA3E0FFE4FBFA7980783E
:1054A50045124F58C004C005C006C007E4FFFE7D85
:1054B500A07C419004A6E0F8A3E0F9A3E0FAA3E0FC
:1054C500FB124E4FD003D002D001D000124E4FD068
:1054D50003D002D001D000124D5E90042212525C1E
:1054E5009005A7E0FCA3E0FDA3E0FEA3E0FFC00458
:1054F500C005C006C0079004C5E0FEA3E07802C35E
:1055050033CE33CED8F92428F58274043EF583E0F2
:10551500F8A3E0F9A3E0FAA3E0FBD007D006D00595
:10552500D004124D5E9005A712525C9004C6E004AB
:10553500F070069004C5E004F002544F900422E098
:10554500FCA3E0FDA3E0FEA3E0FFC004C005C00688
:10555500C00790052DE0FCE4125078A804A905AA1F
:1055650006AB07D007D006D005D004124F589004DB
:105575002212525C9005A7E0FCA3E0FDA3E0FEA388
:10558500E0FFC004C005C006C00790052DE0FCE49F
:10559500125078A804A905AA06AB07D007D006D0F3
:1055A50005D004124F589005A712525CE4FFFE7D0A
:1055B500C87C439005A7E0F8A3E0F9A3E0FAA3E0CF
:1055C500FB124FF560025018E4FFFEFDFC9005A7A5
:1055D500E0F8A3E0F9A3E0FAA3E0FB124FF5500AC7
:1055E5009005A71252680000000030060512648D70
:1055F500C2069005A6E070051258F9800A9005A626
:0D560500E0B4010312663512789A0262C308
:1030800030B2030231C29004BFE0FEA3E0FFC39060
:1030900004C2E09F9004C1E09E50030231C290053B
:1030A000ABE0FEA3E0FF9464EE64809480500302E2
:1030B0003143EF946EEE6480948040030231437C90
:1030C000007D0A1251ECEC6003023386ED14602D92
:1030D00014604D24026003023386C39004BDE09463
:1030E000F49004BCE094014003023386A3E004F0B2
:1030F00070069004BCE004F0C202023386C3900460
:10310000B3E094F49004B2E094014003023386A348
:10311000E004F070069004B2E004F0C202023386CC
:10312000C39004B1E094F49004B0E0940140030231
:103130003386A3E004F070069004B0E004F0C2020D
:103140000233869005ABE0FEA3E0FFC394C8EE64B3
:103150008094805003023386EF94D2EE6480948092
:1031600040030233867C007D0A1251ECEC600302BE
:103170003386ED146029046003023386C39004B9DA
:10318000E0945E9004B8E094014003023386A3E02B
:1031900004F070069004B8E004F0C20A023386C35B
:1031A0009004B7E094C89004B6E094004003023362
:1031B00086A3E004F070069004B6E004F0C20A02B0
:1031C000338620B20302338620070302338690053C
:1031D000ABE0FEA3E0FFC39464EE64809480500EE5
:1031E000E004F070069005ABE004F00232F2C3EFA9
:1031F0009464EE648094805003023289EF946EEE02
:103200006480948040030232897C007D0A1251EC74
:10321000EC60030232F2ED14602D14604D24026064
:10322000030232F2C39004BDE094F49004BCE09435
:103230000140030232F2A3E004F070069004BCE007
:1032400004F0C2020232F2C39004B3E094F490049A
:10325000B2E0940140030232F2A3E004F070069061
:1032600004B2E004F0C2020232F2C39004B1E0946E
:10327000F49004B0E094015079A3E004F07006905B
:1032800004B0E004F0C20280699005ABE0FEA3E068
:10329000FFC394C8EE648094804057EF94D2EE64EC
:1032A000809480504D7C007D0A1251ECEC7043ED0F
:1032B00014602204703CC39004B9E0945E9004B89A
:1032C000E09401502DA3E004F070069004B8E004EF
:1032D000F0C20A801DC39004B7E094C89004B6E021
:1032E0009400500EA3E004F070069004B6E004F0E1
:1032F000C20A900427E02401FFE433FE9005ABE00E
:10330000FCA3E0FDB5070EECB5060A9005ABE4F0B2
:10331000A304F080689004BEE0FF240AFBE433FAC3
:10332000EDB50314ECB50210C39005ACE09FF0902E
:1033300005ABE09400F0804590052CE0F92414FFE3
:10334000E433FE9005ABE0FCA3E0FDB50706ECB569
:1033500006028019900421E0241EFFE433FE90054C
:10336000ABE0FCA3E0FDB50714ECB50610E9FFC324
:10337000ED9FFEEC94009005ABF0A3CEF0E490043A
:10338000C1F0A3F0C20730B3030234B09004BFE031
:10339000FEA3E0FFC39004C4E09F9004C3E09E50EE
:1033A000030234B09005ABE0FEA3E0FF9464EE644A
:1033B0008094805003023438EF946EEE64809480E1
:1033C00050767C007D0A1251ECEC6003023625ED4C
:1033D00014602614603F24026003023625D3900453
:1033E000BDE094009004BCE094005003023625A395
:1033F000E024FFF09004BC8036D39004B3E0940046
:103400009004B2E094005003023625A3E024FFF0BC
:103410009004B2801AD39004B1E094009004B0E01C
:1034200094005003023625A3E024FFF09004B0E09E
:1034300034FFF0C2020236259005ABE0FEA3E0FFA8
:10344000C394C8EE648094805003023625EF94D272
:10345000EE6480948040030236257C007D0A125180
:10346000ECEC6003023625ED1460220460030236A2
:1034700025D39004B9E094C89004B8E094005003B8
:10348000023625A3E024FFF09004B8801AD39004FC
:10349000B7E094009004B6E094005003023625A3F0
:1034A000E024FFF09004B6E034FFF0C20A023625B3
:1034B00020B3030236252008030236259005ABE031
:1034C000FEA3E0FFC39464EE64809480500EE02479
:1034D000FFF09005ABE034FFF00235C6C3EF946413
:1034E000EE64809480407CEF946EEE648094805013
:1034F000727C007D0A1251ECEC60030235C6ED14BB
:10350000602614603F240260030235C6D39004BDD8
:10351000E094009004BCE0940050030235C6A3E0A0
:1035200024FFF09004BC8033D39004B3E094009067
:1035300004B2E0940050030235C6A3E024FFF090EB
:1035400004B28017D39004B1E094009004B0E094EA
:10355000004073A3E024FFF09004B0E034FFF0C219
:103560000280639005ABE0FEA3E0FFC394C8EE6465
:103570008094804051EF94D2EE6480948050477CD8
:10358000007D0A1251ECEC703DED14601C047036A5
:10359000D39004B9E094C89004B8E094004027A305
:1035A000E024FFF09004B88017D39004B7E09400B3
:1035B0009004B6E09400400EA3E024FFF09004B61F
:1035C000E034FFF0C20A9005ABE0FEA3E0FF4E70CE
:1035D0000F900427E0FD9005ABE4F0A3EDF0803CF4
:1035E000EF64094E70059004BE80229005ABE0FEAA
:1035F000A3E0FF64134E700C90052CE0FD9005AC29
:10360000E02D8010EF641D4E701290052CE0FF90AD
:1036100005ACE02FF09005ABE03400F0E49004C37B
:10362000F0A3F0C20830B2030236D430B30302363E
:10363000D49004BFE0FEA3E0FFC39004A3E09F90FA
:1036400004A2E09E50030236D42003030236D420A5
:1036500004030236D49005ABE0FEA3E0FF940AEE2B
:103660006480948050519004B6E0FCA3E0FD900487
:1036700008E0FAA3E0FBC39DEA9C5002800F90048F
:10368000B8E0FCA3E0FDD3EB9DEA9C400890040861
:10369000ECF0A3EDF0900410E070047D0180027D59
:1036A00000900410EDF0C205E49005ABF0A3F0C269
:1036B00000C2B4C20380127C007D0A1251EC900556
:1036C000ABEEF0A3EFF0C203E49004A2F0A3F0C2CB
:1036D0000402388620B30302388620B203023886FB
:1036E0002003030238869004BFE0FEA3E0FFC390EE
:1036F00004A3E09F9004A2E09E40030238862004C9
:1037000003023886900427E0FF9005ABE0FCA3E0BD
:10371000FD6F7001EC705A9004B6E0FEA3E0FF90DC
:103720000408E0FAA3E0FBC39FEA9E5002800F90DA
:1037300004B8E0FEA3E0FFD3EB9FEA9E40089004AC
:1037400008EEF0A3EFF0900410E070047F01800217
:103750007F00900410EFF0C205E49005ABF0A3F0F9
:10376000C200C2B4C2039004A2F0A3F0C2040238A3
:103770007DC3ED9464EC64809480402D9005ABE0B3
:10378000FEA3E0FF7C007D0A1251ECAA04AB059079
:1037900005ABE0FEA3E0FF7C007D0A1251ECEF2BAD
:1037A000FFEE3A9005AB0238449005ABE0FEA3E093
:1037B000FF640D4E6006EF64164E70159005ABE089
:1037C000FEA3E0FF7C007D0A1251EC9005ABEE8079
:1037D000739005ABE0FEA3E0FFC3940AEE6480940F
:1037E00080500D7C007D0A1251859005ABEE80540F
:1037F0009005ABE0FEA3E0FFC3941EEE64809480CE
:103800004048EF9428EE64809480503E7C007D0A0E
:103810001251EC900421E024FFFFE434FFFEED6F31
:103820007002EC6E600BAF059005A6EFF0C2018050
:103830004C9005ABE0FEA3E0FF7C007D0A1251EC4A
:103840009005ABEEF0A3EFF080339005ABE0FEA364
:10385000E0FF7C007D0A1251EC7C007D64125185F2
:10386000AA06AB079005ABE0FEA3E0FF7D0A12516C
:10387000ECEB2DFEEA3C9005ABF0A3CEF0C203E4E6
:103880009004A2F0A3F020B30302398720B2030210
:103890003987E49004A2F0A3F0C203D2042002729C
:1038A0009004BCE0FEA3E090040AF0EEA3F09004C4
:1038B000B2E0FEA3E0900406F0EEA3F09004B0E0C6
:1038C000FEA3E0900404F0EEA3F07F007E021279E4
:1038D000447B017A04790A9005BAE4F0A37402F0FB
:1038E0007F00FE1277347B017A0479069005BAE4F2
:1038F000F0A37402F07F04FE1277347B017A04791E
:10390000049005BAE4F0A37402F07F08FE12773445
:10391000D202200A519004B8E0FEA3E09005B1F075
:10392000EEA3F09004B6E0FEA3E09005AFF0EEA3A6
:10393000F07F007E041279447B017A0579B190050D
:10394000BAE4F0A37402F07F007E041277347B01A6
:103950007A0579AF9005BAE4F0A37402F07404FF1D
:10396000FE127734D20A20011E7F007E06127944AF
:103970007B017A0579A69005BAE4F0A304F07F00F4
:0D3980007E06127734D201200502D2052206
:102760001278D0123080C39005ACE0940A9005AB8B
:10277000E06480948050639005C37430F0A374FFCC
:10278000F0A3740DF0A3742AF07B117D017F6D120C
:102790006DB69005C37430F0A374FFF0A3740CF011
:1027A000A374C4F07B117D017F02126DB69005C346
:1027B0007440F09005ACE07F00FEEF24C4F974078C
:1027C0003EFA9005C474FFF0A3EAF0A3E9F07B2081
:1027D000E4FD7F30126DB602307D9005ABE0FEA3C4
:1027E000E0FFC3940AEE64809480500302299AEFBC
:1027F0009414EE64809480400302299A9005C37477
:1028000030F0A374FFF0A3740DF0A3742AF07B11D1
:102810007D017F6D126DB69005C37430F0A374FF17
:10282000F0A3740CF0A374C4F07B117D017F02123D
:102830006DB69005ABE0FEA3E0FF7C007D0A12516F
:10284000EC7E007FD812518574A42FF974173EFADC
:102850009005C474FFF0A3EAF0A3E9F09005C374F7
:1028600020F07B36E4FD7F34126DB69005ABE0FEC0
:10287000A3E0FF7C007D0A1251EC9004BEE024FF2F
:10288000FFE434FFFEC3ED9FEE6480F8EC648098B3
:1028900050107E007FC412518574842FF974113E4C
:1028A000802F9005ABE0FEA3E0FF7C007D0A125173
:1028B000EC9004BEE0FF24FFFBE434FFFAEDB50327
:1028C0002CECB50228EF75F0C4A424B0F9740D35D2
:1028D000F0FA9005C474FFF0A3EAF0A3E9F09005C4
:1028E000C37438F07B1CE4FD7F16126DB6E49004CF
:1028F000C5F0A3F09004BEE0FF9004C5E0FAA3E0A9
:10290000FBC39FEA9400400302307D9005ABE0FEDC
:10291000A3E0FF7C007D0A1251ECEB6D7002EA6CC3
:102920009004BE602FE024FFFDE434FFFC7E007FB6
:10293000481251979004C5A3E0FEEF8EF0A4241630
:10294000FF9005C37408F0A374FFF0A3740DF0A307
:1029500074F6802DE024FFFDE434FFFC7E007F4808
:102960001251979004C5A3E0FEEF8EF0A42416FF49
:102970009005C37408F0A374FFF0A3740EF0A37461
:1029800002F07B0C7D07126DB69004C6E004F07077
:10299000069004C5E004F00228F49005ABE0FEA325
:1029A000E0FFC39414EE648094805003022B5AEF2E
:1029B000941EEE648094804003022B5A9005C374E9
:1029C00030F0A374FFF0A3740DF0A3742AF07B1110
:1029D0007D017F6D126DB69005C37430F0A374FF56
:1029E000F0A3740CF0A374C4F07B117D017F02127C
:1029F0006DB69005ABE0FEA3E0FF7C007D0A1251AE
:102A0000EC7E007FD812518574042FF9741B3EFAB6
:102A10009005C474FFF0A3EAF0A3E9F09005C37435
:102A200020F07B36E4FD7F34126DB69005ABE0FEFE
:102A3000A3E0FF7C007D0A1251EC90052CE024FFFE
:102A4000FFE434FFFEC3ED9FEE6480F8EC648098F1
:102A5000500F7E007FC4125185741C2FF9741680AC
:102A60002F9005ABE0FEA3E0FF7C007D0A1251EC45
:102A700090052CE024FFFFE434FFFEEDB5072EECBB
:102A8000B5062A7E007FC412518574D02FF97413C5
:102A90003EFA9005C474FFF0A3EAF0A3E9F09005B4
:102AA000C37438F07B1CE4FD7F16126DB6E490040D
:102AB000C5F0A3F090052CE0FF9004C5E0FAA3E078
:102AC000FBC39FEA9400400302307D9005ABE0FE1B
:102AD000A3E0FF7C007D0A1251ECEB6D7002EA6C02
:102AE00090052C602FE024FFFDE434FFFC7E007F86
:102AF000481251979004C5A3E0FEEF8EF0A424166F
:102B0000FF9005C37408F0A374FFF0A3740DF0A345
:102B100074F6802DE024FFFDE434FFFC7E007F4846
:102B20001251979004C5A3E0FEEF8EF0A42416FF87
:102B30009005C37408F0A374FFF0A3740EF0A3749F
:102B400002F07B0C7D07126DB69004C6E004F070B5
:102B5000069004C5E004F0022AB49005ABE0FEA3A1
:102B6000E0FFC3941EEE648094805003022D21D3B5
:102B7000EF9428EE648094804003022D219005C3D9
:102B80007430F0A374FFF0A3740DF0A3742AF07BEB
:102B9000117D017F6D126DB69005C37430F0A37482
:102BA000FFF0A3740CF0A374C4F07B117D017F02CD
:102BB000126DB69005ABE0FEA3E0FF7C007D0A122B
:102BC00051EC7E007FD812518574602FF974213E3C
:102BD000FA9005C474FFF0A3EAF0A3E9F09005C3EE
:102BE0007420F07B36E4FD7F34126DB69005ABE0C7
:102BF000FEA3E0FF7C007D0A1251EC900421E0244A
:102C0000FFFFE434FFFEEDB50708ECB506047E00D7
:102C1000801C9005ABE0FEA3E0FF7C007D0A125112
:102C2000EC9005A6E07E00B50511EEB5040D7FC45D
:102C3000125185748C2FF9741D801C9005ABE0FE39
:102C4000A3E0FF7C007D0A1251EC7E007FC412518C
:102C50008574D82FF9741F3EFA9005C474FFF0A351
:102C6000EAF0A3E9F09005C37438F07B1CE4FD7F23
:102C700016126DB6E49004C5F0A3F0900421E0FFB5
:102C80009004C5E0FAA3E0FBC39FEA94004003026E
:102C9000307D9005ABE0FEA3E0FF7C007D0A125181
:102CA000ECEB6D7002EA6C900421602FE024FFFDD4
:102CB000E434FFFC7E007F481251979004C5A3E0E6
:102CC000FEEF8EF0A42416FF9005C37408F0A374E1
:102CD000FFF0A3740DF0A374F6802DE024FFFDE453
:102CE00034FFFC7E007F481251979004C5A3E0FE9C
:102CF000EF8EF0A42416FF9005C37408F0A374FFB0
:102D0000F0A3740EF0A37402F07B0C7D07126DB675
:102D10009004C6E004F070069004C5E004F0022CB4
:102D20007B9005ABE0FEA3E0FFC39464EE64809467
:102D3000805003022ED3EF946EEE648094804003A3
:102D4000022ED39005C37430F0A374FFF0A3740E69
:102D5000F0A3740EF07B117D017F6D126DB69005AE
:102D6000C37430F0A374FFF0A3740DF0A37490F05B
:102D70007B117D017F02126DB69005ABE0FEA3E0F2
:102D8000FF7C007D0A1251EC7E007FC412518574D5
:102D9000742FF9740E3EFA9005C474FFF0A3EAF0A4
:102DA000A3E9F09005C37438F07B1CE4FD7F161294
:102DB0006DB69005ABE0FEA3E0FF7C007D0A1251EA
:102DC000EC7E007FD812518574A42FF974173EFA57
:102DD0009005C474FFF0A3EAF0A3E9F09005C37472
:102DE00020F07B36E4FD7F34126DB69005ABE0FE3B
:102DF000A3E0FF7C007D0A1251ECEC7029ED146019
:102E00000C14600E2402701E9004BC80089004B262
:102E100080039004B0E0FAA3E0FB9005B97404F0DD
:102E2000FD7F351260C8E49004C5F0A3F09004BEA5
:102E3000E0FF9004C5E0FAA3E0FBC39FEA940040E2
:102E40000302307D9005ABE0FEA3E0FF7C007D0A2D
:102E50001251ECEB6D7002EA6C9004BE602FE0241E
:102E6000FFFDE434FFFC7E007F481251979004C5BB
:102E7000A3E0FEEF8EF0A42416FF9005C37408F0C3
:102E8000A374FFF0A3740DF0A374F6802DE024FF6B
:102E9000FDE434FFFC7E007F481251979004C5A3E7
:102EA000E0FEEF8EF0A42416FF9005C37408F0A393
:102EB00074FFF0A3740EF0A37402F07B0C7D071274
:102EC0006DB69004C6E004F070069004C5E004F00E
:102ED000022E2D9005ABE0FEA3E0FFC394C8EE6484
:102EE000809480500302307DEF94D2EE6480948011
:102EF000400302307D9005C37430F0A374FFF0A34B
:102F0000740EF0A3740EF07B117D017F6D126DB60F
:102F10009005C37430F0A374FFF0A3740DF0A37494
:102F200090F07B117D017F02126DB69005ABE0FE43
:102F3000A3E0FF7C007D0A1251EC7E007FC4125199
:102F40008574D02FF974133EFA9005C474FFF0A372
:102F5000EAF0A3E9F09005C37438F07B1CE4FD7F30
:102F600016126DB69005ABE0FEA3E0FF7C007D0A73
:102F70001251EC7E007FD812518574042FF9741B16
:102F80003EFA9005C474FFF0A3EAF0A3E9F09005BF
:102F9000C37420F07B36E4FD7F34126DB69005AB30
:102FA000E0FEA3E0FF7C007D0A1251ECEC7021ED05
:102FB00014600804701A9004B880039004B6E0FA14
:102FC000A3E0FB9005B97403F07D047F351260C85F
:102FD000E49004C5F0A3F090052CE0FF9004C5E058
:102FE000FAA3E0FBC39FEA9400400302307D900502
:102FF000ABE0FEA3E0FF7C007D0A1251ECEB6D70AC
:1030000002EA6C90052C602FE024FFFDE434FFFC05
:103010007E007F481251979004C5A3E0FEEF8EF02A
:10302000A42416FF9005C37408F0A374FFF0A374E2
:103030000DF0A374F6802DE024FFFDE434FFFC7E48
:10304000007F481251979004C5A3E0FEEF8EF0A4D4
:103050002416FF9005C37408F0A374FFF0A3740E48
:10306000F0A37402F07B0C7D07126DB69004C6E0ED
:1030700004F070069004C5E004F0022FD702789A9D
:1058F9009005A7E0FCA3E0FDA3E0FEA3E0FF1250A2
:10590900ACAB07AA06E4FDFF126F9F900408E0FA0A
:10591900A3E0FB9005B97401F07D037F30126CBCE4
:10592900900422E0FCA3E0FDA3E0FEA3E0FF9005C4
:10593900B712525CE4FD7F30125BCA9004B6E0FCFA
:10594900A3E0FDE41250739005A7E0F8A3E0F9A3E2
:10595900E0FAA3E0FB124FF550030259F59004B8A1
:10596900E0FCA3E0FDE41250739005A7E0F8A3E082
:10597900F9A3E0FAA3E0FB124FF56002506E900420
:10598900B6E0FCA3E0FDE4125073A804A905AA0639
:10599900AB079005A7E0FCA3E0FDA3E0FEA3E0FFB1
:1059A900124D5AE4FBFA79C87842124E4FC004C02E
:1059B90005C006C0079004B6E0FEA3E0FFC390044B
:1059C900B9E09FFD9004B8E09EFCE4125073A8046E
:1059D900A905AA06AB07D007D006D005D004124FF7
:1059E900581250AC9005B8EFF0E4802F9004B8E05D
:1059F900FCA3E0FDE41250739005A7E0F8A3E0F9D9
:105A0900A3E0FAA3E0FB124FF5600B40099005B83B
:105A19007464F0E48005E49005B8F0FB7D067F0826
:105A29001269449004B4E0FCA3E0FDEC12507390B9
:105A3900040CE0F8A3E0F9A3E0FAA3E0FB124FF5A8
:105A4900607A3000779004B4E0FEA3E0FF7C007D2B
:105A59000A1251ECAC06AD07EC12507390040CE03D
:105A6900F8A3E0F9A3E0FAA3E0FB124D5A9004ACC5
:105A790012525C9004ACE0FCA3E0FDA3E0FEA3E0BD
:105A8900FF7BCD7ACC794C783F124E4F9004AC1203
:105A9900525C9004B4E0FEA3E0FF7C007D0A125141
:105AA900ECAC06AD07EC1250739004ACE0F8A3E03F
:105AB900F9A3E0FAA3E0FB124D5A801C20001F90C5
:105AC900040CE0FCA3E0FDA3E0FEA3E0FF7BCD7A9C
:105AD900CC794C783F124E4F90040C12525CE4FF83
:105AE900FE7D807C3F90040CE0F8A3E0F9A3E0FA86
:105AF900A3E0FB124D5E1250AC9005B8EFF07B01AC
:105B09007D067F411269449004B6E0FEA3E0FFC31D
:105B1900900409E09FFF900408E09EFE7C007D64EC
:105B29001251859004B6E0FCA3E0FDC39004B9E0EE
:105B39009DFD9004B8E09CFC125197AB07C00390FF
:105B49000408E0FFA3E09005B8CFF0A3EFF09005BB
:105B5900A7E0FCA3E0FDA3E0FEA3E0FF1250AC9098
:105B690005BAEEF0A3EFF0D0037D307F0B125E9300
:105B79002000139005C37430F0A374FFF0A37407D9
:105B8900F0A374C88030D39004ABE094059004AAC4
:105B9900E0648094809005C37430400EF0A374FFD4
:105BA900F0A37406F0A374CC800CF0A374FFF0A3E7
:105BB9007405F0A374D0F07B2AE4FD7F54126DB60E
:015BC90022B9
:106635009005A7E0FCA3E0FDA3E0FEA3E0FF125058
:10664500ACAB07AA06E49005B9F0FDFF126CBC904F
:106655000408E0FAA3E0FBE49005B9F07D03FF121E
:106665006CBC9005C3741020000EF0A374FFF0A35A
:106675007424F0A37408800CF0A374FFF0A37423B2
:10668500F0A374E8F07B107D067F04126DB69005CB
:10669500C37440F0A374FFF0A37424F0A37428F02E
:1066A5007B67E4FD7F19126DB69004C5E4F0A37411
:1066B5001AF09004C5E0FEA3E0FFC39480EE9400B9
:1066C5005054EF2401FFEF5403703B9004B6E0FEF5
:1066D500A3E0FFC39004B9E09FFB9004B8E09EFAE5
:1066E500900408E0FEA3E0FF7C007D3C125185ADDF
:1066F50003AC02125197C3743C9FFD9004C5A3E0FF
:10670500FF7B011271549004C6E004F070A490045C
:10671500C5E004F0809C200958E49004C5F0A3F07E
:106725009004C5E0FEA3E0FF24C8F58274043EF59D
:1067350083E0FD74C72FF58274043EF583EDF09078
:1067450004C6E004F070069004C5E004F09004C5AA
:10675500E07004A3E0646470C7D2099005A7E0FC6B
:10676500A3E0FDA3E0FEA3E0FF1250AC90052BEFE4
:10677500F0E49004C5F0A3F09004C5E0FAA3E0FBB3
:1067850024C7F58274043AF583E075F03CA4FFAEA6
:10679500F09004B8E0FCA3E0FD125197C3743C9F50
:1067A500FDEB241BFF7B011271549004C6E004F03D
:1067B50070069004C5E004F0C39004C6E0946590AB
:0867C50004C5E0940040B1227C
:10648D00900408E0FCA3E0FDE41250739005A7E032
:10649D00F8A3E0F9A3E0FAA3E0FB124D5A1250ACB9
:1064AD009004AAEEF0A3EFF0FDAC06EC12507312BF
:1064BD0079B2E4FBFA79207841124FF56016401459
:1064CD009004AAE0FEA3E0FF9004BBE02FF090043F
:1064DD00BAE03EF0900402E0FEA3E0FF9004AAE0D3
:1064ED00FAA3E0FBC39FFFEA9E9004A4F0A3EFF094
:1064FD00D39004BBE094F49004BAE064809481409E
:10650D00077401F0A374F4F0C39004BBE0940C90F5
:10651D0004BAE06480947E500774FEF0A3740CF00E
:10652D009004BCE0FCA3E0FDAF03AE02125185D395
:10653D00EF94E8EE9403400F7E037FE8125197909D
:10654D0004AAEEF0A3EFF09004B2E0FAA3E0FB9002
:10655D0004BAE0FEA3E0FFAD03AC02125185D3EF08
:10656D0094E8EE9403400F7E037FE8125197900458
:10657D00BAEEF0A3EFF09004B0E0FAA3E0FB9004C4
:10658D00A4E0FEA3E0FFAD03AC02125185D3EF945E
:10659D00E8EE9403400F7E037FE81251979004BA02
:1065AD00EEF0A3EFF09004BAE0FCA3E0FD9004B28E
:1065BD00E0FEA3E0FF125185AA06AB079004AAE006
:1065CD00FCA3E0FD9004BCE0FEA3E0FF125185EFBB
:1065DD002BFBEE3AFA9004A4E0FCA3E0FD9004B08E
:1065ED00E0FEA3E0FF125185EF2BFFEE3AFE900483
:1065FD00B4F0A3EFF0D394E8EE64809483400A9056
:10660D0004B47403F0A374E8F0C39004B4E06480A0
:10661D0094805004E4F0A3F09004AAE0FFA3E0906E
:08662D000402CFF0A3EFF022FC
:10793100438E805389F0758A66758C7EC28DD28C98
:03794100D2A922A6
:10796800438E0475D78575D6F9438E1043AF04222C
:10791C00E4FDFCC3ED9FEC9E500A0000000DBD0081
:04792C00010C80EFDB
:017930002234
:0E79960075DE20E4F5BDF5BE7F14FE02791CFF
:10739400EE6003027428EFB41000400302742890D6
:1073A40073AAF82828730273DA0273DF0273E40203
:1073B40073E90273EE0273F30273F80273FD02744D
:1073C4000202740702740C02741102741602741B14
:1073D40002742002742575BCC0804975BCC1804408
:1073E40075BCC2803F75BCC3803A75BCC48035751A
:1073F400BCC5803075BCC6802B75BCC7802675BCE7
:10740400C8802175BCC9801C75BCCA801775BCCBEB
:10741400801275BCCC800D75BCCD800875BCCE8047
:107424000375BCCF7F0A7E0012791CE5BC30E5FBF6
:1074340053BCDFAFBDEFFEADBE7C00E42DFFEC3EE0
:02744400FE2226
:086EAD009005B5EEF0A3EFF033
:106EB500FDAC06E41250739005B7E0F8A3E0F9A322
:106EC500E0FAA3E0FB124E4FC004C005C006C007A0
:106ED5009005B5E0FCA3E0FDE4125073D003D002A9
:106EE500D001D000124E4FC004C005C006C00790A7
:106EF50005B5E0FCA3E0FDE4125073D003D002D049
:106F050001D000124E4FC004C005C006C007900551
:106F1500B5E0FCA3E0FDE41250739005BBE0F8A3D7
:106F2500E0F9A3E0FAA3E0FB124E4FC004C005C090
:106F350006C0079005B5E0FCA3E0FDE4125073D050
:106F450003D002D001D000124E4FD003D002D001A1
:106F5500D000124D5EC004C005C006C0079005B53F
:106F6500E0FCA3E0FDE41250739005BFE0F8A3E058
:106F7500F9A3E0FAA3E0FB124E4FD003D002D001F3
:106F8500D000124D5E9005C3E0F8A3E0F9A3E0FA46
:096F9500A3E0FB124D5E1250ACAA
:016F9E0022D0
:10398D000000000000000000002F000000000700F4
:10399D00070000147F147F1400242A7F2A1200626E
:1039AD00640813230036495522500000050300001A
:1039BD0000001C224100000041221C000014083EA2
:1039CD0008140008083E0808000000A06000000868
:1039DD0008080808000060600000002010080402BC
:1039ED00003E5149453E0000427F4000004261517A
:1039FD004946002141454B31001814127F10002714
:103A0D0045454539003C4A494930000171090503D6
:103A1D0000364949493600064949291E0000363607
:103A2D00000000005636000000081422410000146A
:103A3D001414141400004122140800020151090647
:103A4D0000324959513E007C1211127C007F4949C8
:103A5D004936003E41414122007F4141221C007FF9
:103A6D0049494941007F09090901003E4149497A07
:103A7D00007F0808087F0000417F41000020404181
:103A8D003F01007F08142241007F40404040007FED
:103A9D00020C027F007F0408107F003E4141413E31
:103AAD00007F09090906003E4151215E007F091979
:103ABD0029460046494949310001017F0101003F76
:103ACD004040403F001F2040201F003F4038403FF6
:103ADD00006314081463000708700807006151495A
:103AED00454300007F41410000552A552A550000ED
:103AFD0041417F0000013E4141222060FF602000D6
:103B0D002060FF602000002054545478007F48440A
:103B1D00443800384444442000384444487F003839
:103B2D005454541800087E0901020018A4A4A47C62
:103B3D00007F080404780000447D4000004080842C
:103B4D007D00007F102844000000417F4000007C74
:103B5D0004180478007C0804047800384444443880
:103B6D0000FC242424180018242418FC007C0804CC
:103B7D00040800485454542000043F444020003CA5
:103B8D004040207C001C2040201C003C4030403C2C
:103B9D00004428102844001CA0A0A07C00446454BC
:103BAD004C44141414141414000000000000000000
:103BBD000000000000000000000000F80000000000
:103BCD00000000333000000000100C06100C060041
:103BDD00000000000000000040C07840C0784000A8
:103BED00043F04043F040400007088FC083000000A
:103BFD00001820FF211E0000F008F000E018000062
:103C0D0000211C031E211E0000F00888700000001A
:103C1D001E2123241927211010160E00000000006C
:103C2D000000000000000000000000E01804020089
:103C3D00000000071820400000020418E0000000FA
:103C4D000040201807000000404080F080404000F8
:103C5D000202010F01020200000000F0000000004E
:103C6D000101011F01010100000000000000000022
:103C7D0080B0700000000000000000000000000097
:103C8D000001010101010101000000000000000020
:103C9D000000000000000303000000008060180415
:103CAD00006018060100000000E010080810E00098
:103CBD00000F102020100F00001010F80000000061
:103CCD000020203F202000000070080808887000A8
:103CDD000030282422213000003008888848300028
:103CED000018202020110E000000C02010F8000048
:103CFD0000070424243F240000F8088888080800E1
:103D0D000019212020110E0000E0108888180000F5
:103D1D00000F112020110E0000380808C8380800C7
:103D2D000000003F00000000007088080888700047
:103D3D00001C222121221C0000E010080810E000C8
:103D4D000000312222110F00000000C0C000000051
:103D5D000000003030000000000000800000000076
:103D6D00000080600000000000008040201008006E
:103D7D000001020408102000404040404040400037
:103D8D000404040404040400000810204080000012
:103D9D000020100804020100007048080808F00017
:103DAD000000003036010000C030C828E810E000E7
:103DBD000718272423140B000000C038E000000072
:103DCD00203C23020227382008F8888888700000DC
:103DDD00203F202020110E00C030080808083800B0
:103DED00071820202010080008F808080810E00027
:103DFD00203F202020100F0008F88888E8081000C8
:103E0D00203F20202320180008F88888E80810009B
:103E1D00203F200003000000C030080808380000D3
:103E2D0007182020221E020008F808000008F808D4
:103E3D00203F210101213F20000808F8080800005B
:103E4D000020203F2020000000000808F80808008E
:103E5D00C08080807F00000008F888C02818080006
:103E6D00203F20012638200008F80800000000003F
:103E7D00203F20202020300008F8F800F8F8080036
:103E8D00203F003F003F200008F830C00008F80830
:103E9D00203F200007183F00E01008080810E00040
:103EAD000F10202020100F0008F808080808F00057
:103EBD00203F210101010000E01008080810E0007A
:103ECD000F18242438504F0008F88888888870000F
:103EDD00203F2000030C30200070880808083800AF
:103EED000038202121221C00180808F808081800A5
:103EFD000000203F2000000008F808000008F80826
:103F0D00001F202020201F000878880000C83808D6
:103F1D00000007380E010000F80800F80008F8004E
:103F2D00033C0700073C03000818688080681808E8
:103F3D0020302C03032C30200838C800C838080066
:103F4D000000203F2000000010080808C8380800B5
:103F5D002038262120201800000000FE0202020059
:103F6D000000007F40404000000C30C00000000009
:103F7D00000000010638C00000020202FE00000031
:103F8D00004040407F0000000000040202020400D7
:103F9D000000000000000000000000000000000014
:103FAD0080808080808080800002020400000000FC
:103FBD0000000000000000000000808080800000F4
:103FCD000019242222223F2008F8008080000000E2
:103FDD00003F112020110E000000008080800000A5
:103FED00000E112020201100000000808088F800B4
:103FFD00000E112020103F200000808080800000E6
:10400D00001F222222221300008080F08888881849
:10401D000020203F20200000000080808080800054
:10402D00006B94949493600008F8008080800000E9
:10403D00203F210000203F200080989800000000C4
:10404D000020203F202000000000008098980000F4
:10405D0000C08080807F000008F800008080800014
:10406D00203F24022D302000000808F80000000039
:10407D000020203F202000008080808080808000F4
:10408D00203F20003F20003F808000808080000086
:10409D00203F210000203F20000080808080000014
:1040AD00001F202020201F00808000808000000045
:1040BD0080FFA12020110E00000000808080800074
:1040CD00000E112020A0FF80808080008080800065
:1040DD0020203F2120000100000080808080800092
:1040ED000033242424241900008080E08080000007
:1040FD000000001F20200000808000000080800054
:10410D00001F202020103F208080800000808080B4
:10411D0000010E3008060100808000800080808044
:10412D000F300C030C300F00008080008080800069
:10413D000020312E0E312000808080000080808094
:10414D0080818E7018060100008080808080800044
:10415D000021302C2221300000000000807C020262
:10416D0000000000003F404000000000FF00000084
:10417D0000000000FF0000000002027C8000000033
:10418D000040403F00000000112244881122448865
:0A419D000101010102020202088084
:1043D8006400000000000000000000000000000071
:1043E80000000000000000000000000000000000C5
:1043F80000000000000000000000000000000000B5
:1044080000000000000000000000000000000000A4
:104418000000000000000000000000000000000094
:0847D80000000000C10DC18CBE
:1078B600EF4E60157D087C07ED1DAA0470011C4A79
:0978C60070F6EF1F70EA1E80E766
:0178CF002296
:10787E009005B5EFF07006FD7FA61277A99005B5BD
:0C788E00E0B40107E4FD7FA71277A922F7
:1077D0009005B5EFF0700DFD7FC81277A9E4FD7F2D
:1077E000A11277A99005B5E0B4010EE4FD7FC012A7
:0A77F00077A9E4FD7FA01277A9221B
:020003000022D9
:0F797800D2B6D2B5120003C2B6120003C2B522B6
:0A79CB00C2B6D2B5120003D2B622F4
:0F798700D2B6120003D2B5120003C2B50200033C
:10781F00E4FEC2B5EF30E704D2B68002C2B6120062
:10782F0003D2B5120003C2B5EF25E0FF0EEEB40888
:01783F00E167
:017840002225
:0A779F001277A9E4FF1277A97F100A
:1077A900AC071279787F7812781F127987ED600417
:1077B9007F408002E4FF12781F127987AF041278A4
:0777C9001F1279870279CB42
:10786000AB07ED24B0FFE4FD1277A9EB54F0C4544C
:0E7870000F4410FF1277A9EB540FFF0277A907
:10795700E4FD7F8D1277A97F141277A97FAF027795
:01796700A976
:0C79BF00E4FD7F8D1277A47FAE0277A953
:10784100E4FBEB24B0FFE4FD12779FE4FA7D01E451
:0E785100FF1277A90AEAB480F40BEBB408E446
:01785F002206
:086BB4009005DAEFF0A3EDF00B
:106BBC009005DDE0FFC313F9A3F0E4A3F0A3F0EF1D
:106BCC00B40809A3E4F0A37406F0802F9005DDE06F
:106BDC00FF131313541FFD7C00EF54077E00600459
:106BEC007F0180027F00EF2DFFEE3CFEE9FD7C0073
:106BFC001251859005E1EEF0A3EFF0EB24E0FA9052
:106C0C0005DAE0FFA3E0FD127860E49005DFF0A365
:106C1C00F09005E1E0FEA3E0FFC39005E0E09F905B
:106C2C0005DFE09E4003026CBB9005DEE0FD7C00BE
:106C3C00A3E0FEA3E0FF125197ED4C70159005DD1B
:106C4C00E06408600D9005DAE0FFA3E0FD04F012AB
:106C5C0078609005DDE0FBB408179005DFE0FEA33B
:106C6C00E0FF75F006EAA4248DF582E5F034398056
:106C7C0019EBB4103A9005DFE0FEA3E0FF75F010BD
:106C8C00EAA424B5F582E5F0343BF583E5822FF5D3
:106C9C0082E5833EF583E493FF7D011277A990058D
:0F6CAC00E0E004F070069005DFE004F0026C1DDC
:016CBB0022B6
:0777FA00C3EF9E14FD7F0A9E
:07780100900602EFF0A9055B
:107808007F017E00AD0119ED600C900602E0FD7C61
:067818000012518580EE14
:01781E002247
:0E7076009005D0EFF0A3EDF0A3EAF0A3EBF04D
:10708400E49005D8F0A3F09005D5E0B40806900587
:10709400D87402F0E49005D6F09005D4E0FF900592
:1070A400D6E0FEC39F40030271491277FA9005D2DD
:1070B400E0FCA3E0FDCFCDCFCECCCE1251977C0027
:1070C4007D0A1251979005D7EDF09005D9E0703CF8
:1070D4009005D4E014FF9005D6E0FEC39F502DA385
:1070E400E070239005D5E0FCC313FF9005D8E02F92
:1070F4008EF0A4FF9005D0E02FFFA3E0FD9005DD06
:10710400ECF07B2080339005D97401F09005D5E034
:10711400FEC313FF9005D8E02FFF9005D6E0FDEFE6
:107124008DF0A4FF9005D0E02FFFA3E0FD9005D7DC
:10713400E02430FB9005DDEEF0126BB49005D6E050
:0571440004F002709D43
:017149002223
:107688009005EBEFF0A3EDF0A3EBF0A3EAF0A3E98C
:01769800F001
:10769900E49005F1F09005EDE0FBA3E0FAA3E0F931
:1076A9009005F1E0F582758300125146604090051E
:1076B900EBE0FFA3E0FD9005F1E0FE04F08E82759A
:1076C9008300125146FB9005F0E09005DDF0126B46
:1076D900B49005F0E0FFB408099005EBE02406F04A
:0E76E90080B3EFC313FF9005EBE02FF080A7F6
:0176F7002270
:10721B009005B5EEF0A3EFF0A3ECF0A3EDF0A3EB2C
:01722B00F072
:10722C00E49005BEF0A3F09005BAE0FF13131354DD
:10723C001FFEEF540760047F0180027F00EE2F9049
:10724C0005BAF0E49005C0F0A3F09005BAE0FF9009
:10725C0005C0E0FCA3E0FDC39F7480F8EC6480984B
:10726C0050709005B5A3E0FFA3A3E0FEED2EFD1238
:10727C007860E49005C2F0A3F09005B9E0FFC390EC
:10728C0005C3E09F7480F89005C2E064809850318B
:10729C009005BBE0FBA3E0FAA3E0F9A3E475F001D1
:1072AC0012523885F082F583125146FF7D01127718
:1072BC00A99005C3E004F070C09005C2E004F08012
:1072CC00B89005C1E004F070819005C0E004F002B4
:0272DC007256E8
:0172DE00228D
:10744600C2A37FC87E001278B6D2A37FC87E001280
:1074560078B6E4FD7FAE12779F7F401277A97F81D1
:107466001277A97FFF1277A97FA11277A97FC81289
:1074760077A97FA61277A97FA81277A97F3F1277EF
:10748600A97FD31277A9E4FF1277A97FD51277A92E
:107496007F801277A97FD91277A97FF11277A97F0A
:1074A600DA1277A97F121277A97FDB1277A97F40BC
:1074B6001277A97F201277A97F021277A97F8D12F2
:1074C60077A97F141277A97FA41277A97FA61277CE
:1074D600A9127841E4FD7FAF1277A9127841E4FF43
:0B74E60012787EE4FF1277D002795785
:0A714A009005BCE0FF9005C0E0FBDB
:0C7154009005CCEBF0AC079005CBEDF003
:1071600020E003E004F09041A6E493FDFF900400CA
:10717000E0FB3395E0FAD3EB9F7480F86A98400601
:10718000E4F0A3E004F09041A5E49375F008A4FFB7
:10719000900401E0FB3395E0FAD3EB9FE5F06480C7
:1071A000F8EA6480984002E4F09005CBE0131313F2
:1071B000541F8DF0A4AD047C002DFFEC35F0FE745F
:1071C000002FF974003EFA9005CD7401F0A3EAF0A7
:1071D000A3E9F09005CBE05407FF7401A8070880ED
:1071E00002C333D8FCFF9005CCE07017A3E0FBA3EB
:1071F000E475F001125238A9F0FA12512DFEEFF4A5
:107200005E80149005CDE0FBA3E475F001125238C6
:0A721000A9F0FA12512D4F1251732C
:01721A002251
:0B76F8009005F2EBF0A3EAF0A3E9F02C
:1077030012512DFF9005F5E0FBA3E0FAA3E0F91277
:10771300512DFE9005F2E0FBA3E0FAA3E0F9EE128F
:1077230051739005F5E0FBA3E0FAA3E0F9EF0251F2
:0177330073E2
:105612009005BDEDF09005BCEFF0F99005BEEBF002
:10562200E4FA9005C1F0A3F0A31252680000000052
:105632009005C712526800000000E9D39B402690F3
:1056420005BEE0FA9005BCE09005BEF09005BCEA0C
:10565200F09005BFE0FA9005BDE09005BFF090051F
:10566200BDEAF0E4FA9005BDE0FD9005BFE0FEC39F
:105672009D9005C1F09005BCE0FF9005BEE0C39F80
:105682009005C2F0704DEDD39E501C9005BFE0FF17
:105692009005BDE0FDD39F40030258F812714A9075
:1056A20005BDE004F080E49005BFE0FF9005BDE099
:1056B200D39F50030258F89005BDE0FF9005BFE06C
:1056C200FDD39F40030258F812714A9005BFE004CF
:1056D200F080E49005C1E0701F9005BEE0FE9005E9
:1056E200BCE0FFD39E40030258F8A3E0FD12714FC5
:1056F2009005BCE004F080E19005C2E0FC12507815
:10570200C004C005C006C0079005C1E0FC12507875
:10571200D003D002D001D000124F589005C31252CC
:105722005C9005BEE0FCE41250789005C3E0F8A35B
:10573200E0F9A3E0FAA3E0FB124E4FC004C005C09B
:1057420006C0079005BFE0FCE4125078D003D002F7
:10575200D001D000124D5A9005C712525CE4FFFEF0
:105762007D807CBF9005C3E0F8A3E0F9A3E0FAA333
:10577200E0FB124FF5600840067F01C00780047FFE
:1057820000C007E4FFFE7D807C3F9005C3E0F8A3E4
:10579200E0F9A3E0FAA3E0FB124FF550047E01808A
:1057A200027E00D0E05E60529005BEE0FF9005BC34
:1057B200E0D39F40030258F8E0FCFFC007E4125018
:1057C200789005C3E0F8A3E0F9A3E0FAA3E0FB12A6
:1057D2004E4F9005C7E0F8A3E0F9A3E0FAA3E0FB7F
:1057E200124D5E1250ACAD079005C0E0FBD007121F
:1057F20071549005BCE004F080AEE4FFFE7D807C35
:10580200BF9005C3E0F8A3E0F9A3E0FAA3E0FB121E
:105812004FF5600250067F01C00780047F00C00779
:10582200E4FFFE7D807C3F9005C3E0F8A3E0F9A38E
:10583200E0FAA3E0FB124FF540047E0180027E00F5
:10584200D0E04E70030258F89005BFE0FF9005BD0E
:10585200E0D39F504A9005BFE0FF9005BDE0FCD326
:105862009F40030258F8E41250789005C7E0F8A36D
:10587200E0F9A3E0FAA3E0FB124D5A9005C3E0F869
:10588200A3E0F9A3E0FAA3E0FB124F581250AC9048
:1058920005BDE0FD12714F9005BDE004F080B690A9
:1058A20005BFE0FF9005BDE0D39F404A9005BDE0F3
:1058B200FF9005BFE0FCD39F503CE4125078900566
:1058C200C7E0F8A3E0F9A3E0FAA3E0FB124D5A9077
:1058D20005C3E0F8A3E0F9A3E0FAA3E0FB124F58F6
:1058E2001250AC9005BFE0FDA3E0FB12715490058D
:0658F200BFE004F080B6E7
:0158F800228D
:10789A009005BA7440F0A37401F0A37400F0A374C5
:0C78AA0000F07B80E4FDFCFFFE02721B7E
:1078D0009041A5E493FFA3E4938FF0A4FFAEF07D65
:0A78E000007B017A00790002529942
:1067CD009005F8EBF0A3EAF0A3E9F0300C1D90056D
:1067DD00F8E0FBA3E0FAA3E0F9300D0812512DFF0C
:1067ED00EDF4805F12512D4D026940200D030268BA
:1067FD00A7300E539005F8E0FBA3E0FAA3E0F912E1
:10680D00512DFF9005FCE0FEC374089EFE74FFA899
:10681D0006088002C333D8FCFEEDF44E5F125173AF
:10682D009005F8E0FBA3E0FAA3E0F912512DFF90DB
:10683D0005FCE0FE74FFA806088002C313D8FCFE19
:10684D00EDF45E4F0269409005F8E0FBA3E0FAA37A
:10685D00E0F912512DFF9005FCE0FEC374089EFE79
:10686D0074FFA806088002C313D8FCFEEDF44E5F3A
:10687D001251739005F8E0FBA3E0FAA3E0F9125171
:10688D002DFF9005FCE0FE74FFA806088002C333BF
:10689D00D8FCFEEDF45E4F026940300E4C9005F8C9
:1068AD00E0FBA3E0FAA3E0F912512DFF9005FCE007
:1068BD00FEC374089EFE74FFA806088002C333D879
:1068CD00FC4D5F1251739005F8E0FBA3E0FAA3E0D5
:1068DD00F912512DFF9005FCE0FE74FFA80608800B
:1068ED0002C313D8FC5D4F804A9005F8E0FBA3E08E
:1068FD00FAA3E0F912512DFF9005FCE0FEC37408D8
:10690D009EFE74FFA806088002C313D8FC4D5F12CB
:10691D0051739005F8E0FBA3E0FAA3E0F912512DB5
:10692D00FF9005FCE0FE74FFA806088002C333D873
:07693D00FC5D4F12517322B3
:0B6A7F009005E4EDF09005E3EFF0FA65
:106A8A00A3E0FE54079005EAF0EB24E09005E5F058
:106A9A00EE131313541FFF9041A6E493FEEF8EF0FA
:106AAA00A4FFEA7C002FFFEC35F0FE74002FF97486
:106ABA00003EFA9005E77401F0A3EAF0A3E9F0E4D6
:106ACA009005E5E075F010A424B5F582E5F0343BB5
:106ADA00F583E5822CF582E43583F583E493FF9010
:106AEA0005EAE0FEEFA806088002C333D8FCFF904F
:106AFA0005E6F0FDA3E0FBA3E475F001125238A904
:106B0A00F0FA9005FCEEF0C20E1267CD0CECB40858
:106B1A00AF9005EAE07003026BB39005E4E0FFC3AF
:106B2A0094304003026BB3EF131313541F75F064D0
:106B3A00A4FF9005E3E07C002FFFEC35F0FE7464BF
:106B4A002FF974003EFA9005E77401F0A3EAF0A366
:106B5A00E9F0E49005E5E075F006A4248DF582E5F8
:106B6A00F03439F583E5822CF582E43583F583E444
:106B7A0093FF9005EAE0FEC374089EFEEFA806089C
:106B8A008002C313D8FCFF9005E6F0FDA3E0FBA347
:106B9A00E475F001125238A9F0FA9005FCEEF0D231
:096BAA000E1267CD0CECB406AA32
:016BB30022BF
:0979D500900400EFF0A3EDF02294
:0872DF009005FDEFF0A3EDF0B6
:1072E700E4900601F0900600F09005FFF09005FE8F
:1072F700E0FFA3E0FEC39F40030273881277FA9072
:1073070005FDE0FD7C00CFCDCFCECCCE1251977CD2
:10731700007D0A125197AE05900601E0701B90059B
:10732700FEE014FFA3E0C39F500FEE7006A3E00436
:10733700F080459006017401F0900400E0D364806A
:1073470094DE4007E4F0A3E02408F0900401E0D3C2
:10735700648094B04002E4F0900600E0FF9005FFDF
:10736700E0C39F75F006A4FF900400E02FFFA3E0A1
:10737700FDEE2430FB126A7F9005FFE004F00272F5
:0C738700F49005FEE0FF900400E02FF001
:0173930022D7
:0F6DB6009005C0EFF09005C2EBF09005C1EDF035
:106DC500FF9005C9E4F0A3EFF09005C3E01313139A
:106DD500541FFF9005C1E02FFFE433FEC39005CAA1
:106DE500E09F9005C9E09E4003026EAC9005C0E0AF
:106DF500FF9005C7E4F0A3EFF09005C2E0FF900512
:106E0500C0E0F92FFFE433FE9005C7E0FAA3E0FBED
:106E1500C39FEA9E507D9005C1E0FFC39005CAE07F
:106E25009FFF9005C9E09400FE9005C2E0FD7C003F
:106E3500125185E9FDC3EB9DFDEA9CCD2FFFED3E8B
:106E4500FE9005C4E0FBA3E0FAA3E0F98F828E83F0
:106E5500125146FB9041A6E493FF7E009005C9E0E0
:106E6500FCA3E0FD1251859005C8E02FFF9005C7F2
:106E7500E03EFE74002FF58274003EF583EBF09042
:106E850005C8E004F06003026DFE9005C7E004F05C
:106E9500026DFE9005CAE004F06003026DCE900518
:076EA500C9E004F0026DCE0C
:016EAC0022C3
:0E79A400E4F5C7F5C5F5C675C3FF75C4FF222F
:0778EA00ECF5C3AF058FC4EC
:1078F100A2AF92D5C2AF75C65A75C6A50000A2D572
:0379010092AF2220
:10776D00AD07AC0675C78075F52175C5011278EAB0
:10777D00E5C21251730DBD00010C740129F9E43AF3
:10778D00FA9005BA74FFF5F012522245F070DE0240
:02779D0079A4CD
:10794400AD07AC0675C78075F52175C5031278EAD5
:037954000279A411
:10773400AD07AC0675C78075F52175C502ECF5C3B8
:10774400AF058FC412512DF5C21278F10DBD0001A1
:107754000C740129F9E43AFA9005BA74FFF5F012B1
:09776400522245F070D70279A40D
:104D5700025118E86480F8E933E83360110460F021
:104D6700ED33EC337009E8FCE9FDEAFEEBFF2204C2
:104D770060DED3EB9FEA9EE99DE8C2E78CF0C2F7BD
:104D870095F0400CE8CCF8E9CDF9EACEFAEBCFFB89
:104D97001250E385D0F05804700320D5B3E80470AF
:104DA700075002B2D502512292D5EC0460F7E4CC49
:104DB700C0E0C398F8603B94186008400DD0E0FB52
:104DC7000250FAE4FBFAC9FC8028E830E406E4C99B
:104DD700FBE4CAFCE830E305E4C9CACBFCE85407A6
:104DE7006010F8C3E913F9EA13FAEB13FBEC13FCB1
:104DF700D8F130F52FC3E49CFCEF9BFFEE9AFEED54
:104E070099FDD0E0FBEF4E4D4C701222DB030251AF
:104E17001FEC2CFCEF33FFEE33FEED33FDED30E7F7
:104E2700EB0250FAEF2BFFEE3AFEED39FDD0E0FB37
:104E370050130BBB0003025122ED13FDEE13FEEFDF
:084E470013FFEC13FC0250FA0A
:104E4F00EC4D6011E8497017ED33EC3304600DE45D
:104E5F00FCFFFEFD22E933E8330470F8025118120B
:104E6F0050E358046009E4CC24815006285009020D
:104E7F00512228400302511FC0E0EB4A7044B98011
:104E8F0006D0E0FB02510EEF4E701CBD8008EBFF09
:104E9F00EAFEE9FD80EBE98DF0A4FEE5F0024F3864
:104EAF00E9CDF9EAFEEBFFEF89F0A4FCE5F0CE893E
:104EBF00F0A42EFFE435F0CD89F0A42DFEE435F0FB
:104ECF008067EF4E7005BD80D780C3EF8BF0A4AC29
:104EDF00F0EE8BF0A42CFCE435F0F8EF8AF0A42C64
:104EEF00E5F038FCE433CB8DF0A42CFCE5F03BF877
:104EFF00EE8AF0A42CFCE5F038F8E433CF89F0A467
:104F0F002CFCE5F038CF3400CE89F0A42FFFE5F06C
:104F1F003EFEE433C98DF0A42EFEE5F039CD8AF0C4
:104F2F00A42FFFE5F03EFEE43DFD33D0E0FB50073C
:104F3F000BBB000F025122EC2CFCEF33FFEE33FEC4
:064F4F00ED33FD0250FAF3
:104F5500025122EC5D046005E85904700302511802
:104F65001250E3580460F6EC4860F2EC7004FDFE64
:104F7500FF22C860DB2481C85009C398600250062F
:104F850002511F9850CAF582E9294B4A7005AB8238
:104F950002510E75F0007C1A7880C3EF9BEE9AEDF6
:104FA50099400DC3EF9BFFEE9AFEED99FDE842F0A7
:104FB500DC23ACF0D0E0FFD0E0FED0E0FDAB8220FA
:104FC500E7101BEB60BAEC2CFCEF33FFEE33FEED84
:104FD50033FD0250FAE803F830E705C0F075F0003C
:104FE500EF2FFFEE33FEED33FD40B830E7C280AA68
:104FF50074F8CC6480CCC86480C8F58204604FC363
:10500500EB9FF5F0EA9E42F0E99D42F0E89C45F001
:10501500603C501DE5825FFFE582D313CB5BCBF48B
:105025002B5582FB50280ABA002409B900200880B4
:105035001DE5825BFBE582D313CF5FCFF4C3132F4E
:105045005582FF50090EBE00050DBD00010CC3EBD6
:105055009FF5F0EA9E42F0E99D42F0E89C45F0603C
:0950650007CC4820E701B3EC225E
:10506E0075F020800E75F010800575F0087D007EBD
:10507E00007F003392D530D50312524EEC334010E0
:10508E00EF33FFEE33FEED33FDEC33FCD5F0ED22C6
:0E509E00E5F0247EA2D513CC92E7CDCEFF2202
:1050AC00EDD2E7CD33EC3392D524814006E4FFFEFC
:1050BC00FDFC22FCE4CFCECDCC24E0501174FF805B
:1050CC00EDC3CC13CCCD13CDCE13CECF13CF0470F8
:0750DC00F030D5DE02524E58
:0D79B200ED33EC3360065004EC6480FC22E1
:1050E300E9D2E7C933E833F892D5EDD2E7CD33EC13
:0750F30033FC5002B2D5228C
:1050FA00EC30E7100FBF000C0EBE00080DBD000417
:10510A000BEB6014A2D5EB13FCED92E7FD2274FFC2
:10511A00FCFDFEFF22E480F8A2D574FF13FC7D801B
:03512A00E480EF2F
:0300000002758303
:0C758300787FE4F6D8FD7581210275CAFE
:10512D00BB010689828A83E0225002E722BBFE0280
:09513D00E32289828A83E49322B3
:10514600BB010CE58229F582E5833AF583E022501E
:1051560006E92582F8E622BBFE06E92582F8E22268
:0D516600E58229F582E5833AF583E4932282
:10517300BB010689828A83F0225002F722BBFE011B
:02518300F32215
:10518500EF8DF0A4A8F0CF8CF0A428CE8DF0A42E3E
:02519500FE22F8
:10519700BC000BBE0029EF8DF084FFADF022E4CCFC
:1051A700F875F008EF2FFFEE33FEEC33FCEE9DECC5
:1051B700984005FCEE9DFE0FD5F0E9E4CEFD22ED0B
:1051C700F8F5F0EE8420D21CFEADF075F008EF2F55
:1051D700FFED33FD4007985006D5F0F222C398FD46
:0551E7000FD5F0EA22E3
:1051EC00C2D5EC30E709B2D5E4C39DFDE49CFCEEDE
:1051FC0030E715B2D5E4C39FFFE49EFE125197C36E
:10520C00E49DFDE49CFC800312519730D507C3E468
:06521C009FFFE49EFE224C
:10522200C5F0F8A3E028F0C5F0F8E5821582700217
:065232001583E038F022B4
:10523800A3F8E0C5F025F0F0E58215827002158329
:06524800E0C838F0E82286
:0E524E00C3E49FFFE49EFEE49DFDE49CFC2271
:0C525C00ECF0A3EDF0A3EEF0A3EFF022C5
:10526800A8828583F0D083D08212527F12527F1297
:10527800527F12527FE473E493A3C583C5F0C583BC
:10528800C8C582C8F0A3C583C5F0C583C8C582C890
:0152980022F3
:10529900EF4E6012EF60010EEDBB010B89828A832C
:1052A900F0A3DFFCDEFA2289F05007F709DFFCA939
:0C52B900F022BBFEFCF309DFFCA9F02290
:10758F00027904E493A3F8E493A34003F68001F295
:10759F0008DFF48029E493A3F85407240CC8C333FD
:1075AF00C4540F4420C8834004F456800146F6DFCC
:1075BF00E4800B01020408102040809041A7E47E74
:1075CF00019360BCA3FF543F30E509541FFEE493C1
:1075DF00A360010ECF54C025E060A840B8E493A388
:1075EF00FAE493A3F8E493A3C8C582C8CAC583CAB3
:1075FF00F0A3C8C582C8CAC583CADFE9DEE780BE6B
:0147E00000D8
:00000001FF
